
print by printf.elf:     file format elf32-littlearm

Sections:
Idx Name          Size      VMA       LMA       File off  Algn
  0 .isr_vector   000000c0  08000000  08000000  00010000  2**0
                  CONTENTS, ALLOC, LOAD, READONLY, DATA
  1 .text         00001170  080000c0  080000c0  000100c0  2**2
                  CONTENTS, ALLOC, LOAD, READONLY, CODE
  2 .rodata       0000008c  08001230  08001230  00011230  2**2
                  CONTENTS, ALLOC, LOAD, READONLY, DATA
  3 .ARM.extab    00000000  080012bc  080012bc  0002006c  2**0
                  CONTENTS
  4 .ARM          00000000  080012bc  080012bc  0002006c  2**0
                  CONTENTS
  5 .preinit_array 00000000  080012bc  080012bc  0002006c  2**0
                  CONTENTS, ALLOC, LOAD, DATA
  6 .init_array   00000004  080012bc  080012bc  000112bc  2**2
                  CONTENTS, ALLOC, LOAD, DATA
  7 .fini_array   00000004  080012c0  080012c0  000112c0  2**2
                  CONTENTS, ALLOC, LOAD, DATA
  8 .data         0000006c  20000000  080012c4  00020000  2**2
                  CONTENTS, ALLOC, LOAD, DATA
  9 .bss          000000dc  2000006c  08001330  0002006c  2**2
                  ALLOC
 10 ._user_heap_stack 00000600  20000148  08001330  00020148  2**0
                  ALLOC
 11 .ARM.attributes 00000028  00000000  00000000  0002006c  2**0
                  CONTENTS, READONLY
 12 .debug_info   0000022f  00000000  00000000  00020094  2**0
                  CONTENTS, READONLY, DEBUGGING, OCTETS
 13 .debug_abbrev 00000129  00000000  00000000  000202c3  2**0
                  CONTENTS, READONLY, DEBUGGING, OCTETS
 14 .debug_aranges 00000068  00000000  00000000  000203f0  2**3
                  CONTENTS, READONLY, DEBUGGING, OCTETS
 15 .debug_ranges 00000040  00000000  00000000  00020458  2**3
                  CONTENTS, READONLY, DEBUGGING, OCTETS
 16 .debug_macro  00002138  00000000  00000000  00020498  2**0
                  CONTENTS, READONLY, DEBUGGING, OCTETS
 17 .debug_line   00000a8d  00000000  00000000  000225d0  2**0
                  CONTENTS, READONLY, DEBUGGING, OCTETS
 18 .debug_str    00007f07  00000000  00000000  0002305d  2**0
                  CONTENTS, READONLY, DEBUGGING, OCTETS
 19 .comment      00000050  00000000  00000000  0002af64  2**0
                  CONTENTS, READONLY
 20 .debug_frame  00000af0  00000000  00000000  0002afb4  2**2
                  CONTENTS, READONLY, DEBUGGING, OCTETS

Disassembly of section .text:

080000c0 <__do_global_dtors_aux>:
 80000c0:	b510      	push	{r4, lr}
 80000c2:	4c06      	ldr	r4, [pc, #24]	; (80000dc <__do_global_dtors_aux+0x1c>)
 80000c4:	7823      	ldrb	r3, [r4, #0]
 80000c6:	2b00      	cmp	r3, #0
 80000c8:	d107      	bne.n	80000da <__do_global_dtors_aux+0x1a>
 80000ca:	4b05      	ldr	r3, [pc, #20]	; (80000e0 <__do_global_dtors_aux+0x20>)
 80000cc:	2b00      	cmp	r3, #0
 80000ce:	d002      	beq.n	80000d6 <__do_global_dtors_aux+0x16>
 80000d0:	4804      	ldr	r0, [pc, #16]	; (80000e4 <__do_global_dtors_aux+0x24>)
 80000d2:	e000      	b.n	80000d6 <__do_global_dtors_aux+0x16>
 80000d4:	bf00      	nop
 80000d6:	2301      	movs	r3, #1
 80000d8:	7023      	strb	r3, [r4, #0]
 80000da:	bd10      	pop	{r4, pc}
 80000dc:	2000006c 	.word	0x2000006c
 80000e0:	00000000 	.word	0x00000000
 80000e4:	08001218 	.word	0x08001218

080000e8 <frame_dummy>:
 80000e8:	4b04      	ldr	r3, [pc, #16]	; (80000fc <frame_dummy+0x14>)
 80000ea:	b510      	push	{r4, lr}
 80000ec:	2b00      	cmp	r3, #0
 80000ee:	d003      	beq.n	80000f8 <frame_dummy+0x10>
 80000f0:	4903      	ldr	r1, [pc, #12]	; (8000100 <frame_dummy+0x18>)
 80000f2:	4804      	ldr	r0, [pc, #16]	; (8000104 <frame_dummy+0x1c>)
 80000f4:	e000      	b.n	80000f8 <frame_dummy+0x10>
 80000f6:	bf00      	nop
 80000f8:	bd10      	pop	{r4, pc}
 80000fa:	46c0      	nop			; (mov r8, r8)
 80000fc:	00000000 	.word	0x00000000
 8000100:	20000070 	.word	0x20000070
 8000104:	08001218 	.word	0x08001218

08000108 <strlen>:
 8000108:	2300      	movs	r3, #0
 800010a:	5cc2      	ldrb	r2, [r0, r3]
 800010c:	3301      	adds	r3, #1
 800010e:	2a00      	cmp	r2, #0
 8000110:	d1fb      	bne.n	800010a <strlen+0x2>
 8000112:	1e58      	subs	r0, r3, #1
 8000114:	4770      	bx	lr
	...

08000118 <main>:

extern void initialise_monitor_handles(void);


int main(void)
{
 8000118:	b580      	push	{r7, lr}
 800011a:	af00      	add	r7, sp, #0
	initialise_monitor_handles();
 800011c:	f001 f804 	bl	8001128 <initialise_monitor_handles>

    printf("Hello World\n");
 8000120:	4b02      	ldr	r3, [pc, #8]	; (800012c <main+0x14>)
 8000122:	0018      	movs	r0, r3
 8000124:	f000 f908 	bl	8000338 <puts>

	for(;;);
 8000128:	e7fe      	b.n	8000128 <main+0x10>
 800012a:	46c0      	nop			; (mov r8, r8)
 800012c:	08001230 	.word	0x08001230

08000130 <_sbrk>:
 *
 * @param incr Memory size
 * @return Pointer to allocated memory
 */
void *_sbrk(ptrdiff_t incr)
{
 8000130:	b580      	push	{r7, lr}
 8000132:	b086      	sub	sp, #24
 8000134:	af00      	add	r7, sp, #0
 8000136:	6078      	str	r0, [r7, #4]
  extern uint8_t _end; /* Symbol defined in the linker script */
  extern uint8_t _estack; /* Symbol defined in the linker script */
  extern uint32_t _Min_Stack_Size; /* Symbol defined in the linker script */
  const uint32_t stack_limit = (uint32_t)&_estack - (uint32_t)&_Min_Stack_Size;
 8000138:	4a14      	ldr	r2, [pc, #80]	; (800018c <_sbrk+0x5c>)
 800013a:	4b15      	ldr	r3, [pc, #84]	; (8000190 <_sbrk+0x60>)
 800013c:	1ad3      	subs	r3, r2, r3
 800013e:	617b      	str	r3, [r7, #20]
  const uint8_t *max_heap = (uint8_t *)stack_limit;
 8000140:	697b      	ldr	r3, [r7, #20]
 8000142:	613b      	str	r3, [r7, #16]
  uint8_t *prev_heap_end;

  /* Initialize heap end at first call */
  if (NULL == __sbrk_heap_end)
 8000144:	4b13      	ldr	r3, [pc, #76]	; (8000194 <_sbrk+0x64>)
 8000146:	681b      	ldr	r3, [r3, #0]
 8000148:	2b00      	cmp	r3, #0
 800014a:	d102      	bne.n	8000152 <_sbrk+0x22>
  {
    __sbrk_heap_end = &_end;
 800014c:	4b11      	ldr	r3, [pc, #68]	; (8000194 <_sbrk+0x64>)
 800014e:	4a12      	ldr	r2, [pc, #72]	; (8000198 <_sbrk+0x68>)
 8000150:	601a      	str	r2, [r3, #0]
  }

  /* Protect heap from growing into the reserved MSP stack */
  if (__sbrk_heap_end + incr > max_heap)
 8000152:	4b10      	ldr	r3, [pc, #64]	; (8000194 <_sbrk+0x64>)
 8000154:	681a      	ldr	r2, [r3, #0]
 8000156:	687b      	ldr	r3, [r7, #4]
 8000158:	18d3      	adds	r3, r2, r3
 800015a:	693a      	ldr	r2, [r7, #16]
 800015c:	429a      	cmp	r2, r3
 800015e:	d207      	bcs.n	8000170 <_sbrk+0x40>
  {
    errno = ENOMEM;
 8000160:	f000 f846 	bl	80001f0 <__errno>
 8000164:	0003      	movs	r3, r0
 8000166:	220c      	movs	r2, #12
 8000168:	601a      	str	r2, [r3, #0]
    return (void *)-1;
 800016a:	2301      	movs	r3, #1
 800016c:	425b      	negs	r3, r3
 800016e:	e009      	b.n	8000184 <_sbrk+0x54>
  }

  prev_heap_end = __sbrk_heap_end;
 8000170:	4b08      	ldr	r3, [pc, #32]	; (8000194 <_sbrk+0x64>)
 8000172:	681b      	ldr	r3, [r3, #0]
 8000174:	60fb      	str	r3, [r7, #12]
  __sbrk_heap_end += incr;
 8000176:	4b07      	ldr	r3, [pc, #28]	; (8000194 <_sbrk+0x64>)
 8000178:	681a      	ldr	r2, [r3, #0]
 800017a:	687b      	ldr	r3, [r7, #4]
 800017c:	18d2      	adds	r2, r2, r3
 800017e:	4b05      	ldr	r3, [pc, #20]	; (8000194 <_sbrk+0x64>)
 8000180:	601a      	str	r2, [r3, #0]

  return (void *)prev_heap_end;
 8000182:	68fb      	ldr	r3, [r7, #12]
}
 8000184:	0018      	movs	r0, r3
 8000186:	46bd      	mov	sp, r7
 8000188:	b006      	add	sp, #24
 800018a:	bd80      	pop	{r7, pc}
 800018c:	20005000 	.word	0x20005000
 8000190:	00000400 	.word	0x00000400
 8000194:	20000088 	.word	0x20000088
 8000198:	20000148 	.word	0x20000148

0800019c <Reset_Handler>:

  .section .text.Reset_Handler
  .weak Reset_Handler
  .type Reset_Handler, %function
Reset_Handler:
  ldr   r0, =_estack
 800019c:	480d      	ldr	r0, [pc, #52]	; (80001d4 <LoopForever+0x2>)
  mov   sp, r0          /* set stack pointer */
 800019e:	4685      	mov	sp, r0
/* Call the clock system initialization function.*/
  bl  SystemInit
 80001a0:	e000      	b.n	80001a4 <Reset_Handler+0x8>
 80001a2:	bf00      	nop

/* Copy the data segment initializers from flash to SRAM */
  ldr r0, =_sdata
 80001a4:	480c      	ldr	r0, [pc, #48]	; (80001d8 <LoopForever+0x6>)
  ldr r1, =_edata
 80001a6:	490d      	ldr	r1, [pc, #52]	; (80001dc <LoopForever+0xa>)
  ldr r2, =_sidata
 80001a8:	4a0d      	ldr	r2, [pc, #52]	; (80001e0 <LoopForever+0xe>)
  movs r3, #0
 80001aa:	2300      	movs	r3, #0
  b LoopCopyDataInit
 80001ac:	e002      	b.n	80001b4 <LoopCopyDataInit>

080001ae <CopyDataInit>:

CopyDataInit:
  ldr r4, [r2, r3]
 80001ae:	58d4      	ldr	r4, [r2, r3]
  str r4, [r0, r3]
 80001b0:	50c4      	str	r4, [r0, r3]
  adds r3, r3, #4
 80001b2:	3304      	adds	r3, #4

080001b4 <LoopCopyDataInit>:

LoopCopyDataInit:
  adds r4, r0, r3
 80001b4:	18c4      	adds	r4, r0, r3
  cmp r4, r1
 80001b6:	428c      	cmp	r4, r1
  bcc CopyDataInit
 80001b8:	d3f9      	bcc.n	80001ae <CopyDataInit>

/* Zero fill the bss segment. */
  ldr r2, =_sbss
 80001ba:	4a0a      	ldr	r2, [pc, #40]	; (80001e4 <LoopForever+0x12>)
  ldr r4, =_ebss
 80001bc:	4c0a      	ldr	r4, [pc, #40]	; (80001e8 <LoopForever+0x16>)
  movs r3, #0
 80001be:	2300      	movs	r3, #0
  b LoopFillZerobss
 80001c0:	e001      	b.n	80001c6 <LoopFillZerobss>

080001c2 <FillZerobss>:

FillZerobss:
  str  r3, [r2]
 80001c2:	6013      	str	r3, [r2, #0]
  adds r2, r2, #4
 80001c4:	3204      	adds	r2, #4

080001c6 <LoopFillZerobss>:

LoopFillZerobss:
  cmp r2, r4
 80001c6:	42a2      	cmp	r2, r4
  bcc FillZerobss
 80001c8:	d3fb      	bcc.n	80001c2 <FillZerobss>

/* Call static constructors */
  bl __libc_init_array
 80001ca:	f000 f817 	bl	80001fc <__libc_init_array>
/* Call the application's entry point.*/
  bl main
 80001ce:	f7ff ffa3 	bl	8000118 <main>

080001d2 <LoopForever>:

LoopForever:
  b LoopForever
 80001d2:	e7fe      	b.n	80001d2 <LoopForever>
  ldr   r0, =_estack
 80001d4:	20005000 	.word	0x20005000
  ldr r0, =_sdata
 80001d8:	20000000 	.word	0x20000000
  ldr r1, =_edata
 80001dc:	2000006c 	.word	0x2000006c
  ldr r2, =_sidata
 80001e0:	080012c4 	.word	0x080012c4
  ldr r2, =_sbss
 80001e4:	2000006c 	.word	0x2000006c
  ldr r4, =_ebss
 80001e8:	20000148 	.word	0x20000148

080001ec <ADC_COMP_IRQHandler>:
 * @retval : None
*/
  .section .text.Default_Handler,"ax",%progbits
Default_Handler:
Infinite_Loop:
  b Infinite_Loop
 80001ec:	e7fe      	b.n	80001ec <ADC_COMP_IRQHandler>
	...

080001f0 <__errno>:
 80001f0:	4b01      	ldr	r3, [pc, #4]	; (80001f8 <__errno+0x8>)
 80001f2:	6818      	ldr	r0, [r3, #0]
 80001f4:	4770      	bx	lr
 80001f6:	46c0      	nop			; (mov r8, r8)
 80001f8:	20000000 	.word	0x20000000

080001fc <__libc_init_array>:
 80001fc:	b570      	push	{r4, r5, r6, lr}
 80001fe:	2600      	movs	r6, #0
 8000200:	4d0c      	ldr	r5, [pc, #48]	; (8000234 <__libc_init_array+0x38>)
 8000202:	4c0d      	ldr	r4, [pc, #52]	; (8000238 <__libc_init_array+0x3c>)
 8000204:	1b64      	subs	r4, r4, r5
 8000206:	10a4      	asrs	r4, r4, #2
 8000208:	42a6      	cmp	r6, r4
 800020a:	d109      	bne.n	8000220 <__libc_init_array+0x24>
 800020c:	2600      	movs	r6, #0
 800020e:	f001 f803 	bl	8001218 <_init>
 8000212:	4d0a      	ldr	r5, [pc, #40]	; (800023c <__libc_init_array+0x40>)
 8000214:	4c0a      	ldr	r4, [pc, #40]	; (8000240 <__libc_init_array+0x44>)
 8000216:	1b64      	subs	r4, r4, r5
 8000218:	10a4      	asrs	r4, r4, #2
 800021a:	42a6      	cmp	r6, r4
 800021c:	d105      	bne.n	800022a <__libc_init_array+0x2e>
 800021e:	bd70      	pop	{r4, r5, r6, pc}
 8000220:	00b3      	lsls	r3, r6, #2
 8000222:	58eb      	ldr	r3, [r5, r3]
 8000224:	4798      	blx	r3
 8000226:	3601      	adds	r6, #1
 8000228:	e7ee      	b.n	8000208 <__libc_init_array+0xc>
 800022a:	00b3      	lsls	r3, r6, #2
 800022c:	58eb      	ldr	r3, [r5, r3]
 800022e:	4798      	blx	r3
 8000230:	3601      	adds	r6, #1
 8000232:	e7f2      	b.n	800021a <__libc_init_array+0x1e>
 8000234:	080012bc 	.word	0x080012bc
 8000238:	080012bc 	.word	0x080012bc
 800023c:	080012bc 	.word	0x080012bc
 8000240:	080012c0 	.word	0x080012c0

08000244 <memset>:
 8000244:	0003      	movs	r3, r0
 8000246:	1882      	adds	r2, r0, r2
 8000248:	4293      	cmp	r3, r2
 800024a:	d100      	bne.n	800024e <memset+0xa>
 800024c:	4770      	bx	lr
 800024e:	7019      	strb	r1, [r3, #0]
 8000250:	3301      	adds	r3, #1
 8000252:	e7f9      	b.n	8000248 <memset+0x4>

08000254 <_puts_r>:
 8000254:	b570      	push	{r4, r5, r6, lr}
 8000256:	0005      	movs	r5, r0
 8000258:	000e      	movs	r6, r1
 800025a:	2800      	cmp	r0, #0
 800025c:	d004      	beq.n	8000268 <_puts_r+0x14>
 800025e:	6983      	ldr	r3, [r0, #24]
 8000260:	2b00      	cmp	r3, #0
 8000262:	d101      	bne.n	8000268 <_puts_r+0x14>
 8000264:	f000 fa6e 	bl	8000744 <__sinit>
 8000268:	69ab      	ldr	r3, [r5, #24]
 800026a:	68ac      	ldr	r4, [r5, #8]
 800026c:	2b00      	cmp	r3, #0
 800026e:	d102      	bne.n	8000276 <_puts_r+0x22>
 8000270:	0028      	movs	r0, r5
 8000272:	f000 fa67 	bl	8000744 <__sinit>
 8000276:	4b2d      	ldr	r3, [pc, #180]	; (800032c <_puts_r+0xd8>)
 8000278:	429c      	cmp	r4, r3
 800027a:	d122      	bne.n	80002c2 <_puts_r+0x6e>
 800027c:	686c      	ldr	r4, [r5, #4]
 800027e:	6e63      	ldr	r3, [r4, #100]	; 0x64
 8000280:	07db      	lsls	r3, r3, #31
 8000282:	d405      	bmi.n	8000290 <_puts_r+0x3c>
 8000284:	89a3      	ldrh	r3, [r4, #12]
 8000286:	059b      	lsls	r3, r3, #22
 8000288:	d402      	bmi.n	8000290 <_puts_r+0x3c>
 800028a:	6da0      	ldr	r0, [r4, #88]	; 0x58
 800028c:	f000 fafb 	bl	8000886 <__retarget_lock_acquire_recursive>
 8000290:	89a3      	ldrh	r3, [r4, #12]
 8000292:	071b      	lsls	r3, r3, #28
 8000294:	d502      	bpl.n	800029c <_puts_r+0x48>
 8000296:	6923      	ldr	r3, [r4, #16]
 8000298:	2b00      	cmp	r3, #0
 800029a:	d129      	bne.n	80002f0 <_puts_r+0x9c>
 800029c:	0021      	movs	r1, r4
 800029e:	0028      	movs	r0, r5
 80002a0:	f000 f8aa 	bl	80003f8 <__swsetup_r>
 80002a4:	2800      	cmp	r0, #0
 80002a6:	d023      	beq.n	80002f0 <_puts_r+0x9c>
 80002a8:	2501      	movs	r5, #1
 80002aa:	426d      	negs	r5, r5
 80002ac:	6e63      	ldr	r3, [r4, #100]	; 0x64
 80002ae:	07db      	lsls	r3, r3, #31
 80002b0:	d405      	bmi.n	80002be <_puts_r+0x6a>
 80002b2:	89a3      	ldrh	r3, [r4, #12]
 80002b4:	059b      	lsls	r3, r3, #22
 80002b6:	d402      	bmi.n	80002be <_puts_r+0x6a>
 80002b8:	6da0      	ldr	r0, [r4, #88]	; 0x58
 80002ba:	f000 fae5 	bl	8000888 <__retarget_lock_release_recursive>
 80002be:	0028      	movs	r0, r5
 80002c0:	bd70      	pop	{r4, r5, r6, pc}
 80002c2:	4b1b      	ldr	r3, [pc, #108]	; (8000330 <_puts_r+0xdc>)
 80002c4:	429c      	cmp	r4, r3
 80002c6:	d101      	bne.n	80002cc <_puts_r+0x78>
 80002c8:	68ac      	ldr	r4, [r5, #8]
 80002ca:	e7d8      	b.n	800027e <_puts_r+0x2a>
 80002cc:	4b19      	ldr	r3, [pc, #100]	; (8000334 <_puts_r+0xe0>)
 80002ce:	429c      	cmp	r4, r3
 80002d0:	d1d5      	bne.n	800027e <_puts_r+0x2a>
 80002d2:	68ec      	ldr	r4, [r5, #12]
 80002d4:	e7d3      	b.n	800027e <_puts_r+0x2a>
 80002d6:	3601      	adds	r6, #1
 80002d8:	60a3      	str	r3, [r4, #8]
 80002da:	2b00      	cmp	r3, #0
 80002dc:	da04      	bge.n	80002e8 <_puts_r+0x94>
 80002de:	69a2      	ldr	r2, [r4, #24]
 80002e0:	429a      	cmp	r2, r3
 80002e2:	dc16      	bgt.n	8000312 <_puts_r+0xbe>
 80002e4:	290a      	cmp	r1, #10
 80002e6:	d014      	beq.n	8000312 <_puts_r+0xbe>
 80002e8:	6823      	ldr	r3, [r4, #0]
 80002ea:	1c5a      	adds	r2, r3, #1
 80002ec:	6022      	str	r2, [r4, #0]
 80002ee:	7019      	strb	r1, [r3, #0]
 80002f0:	68a3      	ldr	r3, [r4, #8]
 80002f2:	7831      	ldrb	r1, [r6, #0]
 80002f4:	3b01      	subs	r3, #1
 80002f6:	2900      	cmp	r1, #0
 80002f8:	d1ed      	bne.n	80002d6 <_puts_r+0x82>
 80002fa:	60a3      	str	r3, [r4, #8]
 80002fc:	2b00      	cmp	r3, #0
 80002fe:	da0f      	bge.n	8000320 <_puts_r+0xcc>
 8000300:	0028      	movs	r0, r5
 8000302:	0022      	movs	r2, r4
 8000304:	310a      	adds	r1, #10
 8000306:	f000 f821 	bl	800034c <__swbuf_r>
 800030a:	250a      	movs	r5, #10
 800030c:	1c43      	adds	r3, r0, #1
 800030e:	d1cd      	bne.n	80002ac <_puts_r+0x58>
 8000310:	e7ca      	b.n	80002a8 <_puts_r+0x54>
 8000312:	0022      	movs	r2, r4
 8000314:	0028      	movs	r0, r5
 8000316:	f000 f819 	bl	800034c <__swbuf_r>
 800031a:	1c43      	adds	r3, r0, #1
 800031c:	d1e8      	bne.n	80002f0 <_puts_r+0x9c>
 800031e:	e7c3      	b.n	80002a8 <_puts_r+0x54>
 8000320:	250a      	movs	r5, #10
 8000322:	6823      	ldr	r3, [r4, #0]
 8000324:	1c5a      	adds	r2, r3, #1
 8000326:	6022      	str	r2, [r4, #0]
 8000328:	701d      	strb	r5, [r3, #0]
 800032a:	e7bf      	b.n	80002ac <_puts_r+0x58>
 800032c:	08001260 	.word	0x08001260
 8000330:	08001280 	.word	0x08001280
 8000334:	08001240 	.word	0x08001240

08000338 <puts>:
 8000338:	b510      	push	{r4, lr}
 800033a:	4b03      	ldr	r3, [pc, #12]	; (8000348 <puts+0x10>)
 800033c:	0001      	movs	r1, r0
 800033e:	6818      	ldr	r0, [r3, #0]
 8000340:	f7ff ff88 	bl	8000254 <_puts_r>
 8000344:	bd10      	pop	{r4, pc}
 8000346:	46c0      	nop			; (mov r8, r8)
 8000348:	20000000 	.word	0x20000000

0800034c <__swbuf_r>:
 800034c:	b5f8      	push	{r3, r4, r5, r6, r7, lr}
 800034e:	0005      	movs	r5, r0
 8000350:	000e      	movs	r6, r1
 8000352:	0014      	movs	r4, r2
 8000354:	2800      	cmp	r0, #0
 8000356:	d004      	beq.n	8000362 <__swbuf_r+0x16>
 8000358:	6983      	ldr	r3, [r0, #24]
 800035a:	2b00      	cmp	r3, #0
 800035c:	d101      	bne.n	8000362 <__swbuf_r+0x16>
 800035e:	f000 f9f1 	bl	8000744 <__sinit>
 8000362:	4b22      	ldr	r3, [pc, #136]	; (80003ec <__swbuf_r+0xa0>)
 8000364:	429c      	cmp	r4, r3
 8000366:	d12e      	bne.n	80003c6 <__swbuf_r+0x7a>
 8000368:	686c      	ldr	r4, [r5, #4]
 800036a:	69a3      	ldr	r3, [r4, #24]
 800036c:	60a3      	str	r3, [r4, #8]
 800036e:	89a3      	ldrh	r3, [r4, #12]
 8000370:	071b      	lsls	r3, r3, #28
 8000372:	d532      	bpl.n	80003da <__swbuf_r+0x8e>
 8000374:	6923      	ldr	r3, [r4, #16]
 8000376:	2b00      	cmp	r3, #0
 8000378:	d02f      	beq.n	80003da <__swbuf_r+0x8e>
 800037a:	6823      	ldr	r3, [r4, #0]
 800037c:	6922      	ldr	r2, [r4, #16]
 800037e:	b2f7      	uxtb	r7, r6
 8000380:	1a98      	subs	r0, r3, r2
 8000382:	6963      	ldr	r3, [r4, #20]
 8000384:	b2f6      	uxtb	r6, r6
 8000386:	4283      	cmp	r3, r0
 8000388:	dc05      	bgt.n	8000396 <__swbuf_r+0x4a>
 800038a:	0021      	movs	r1, r4
 800038c:	0028      	movs	r0, r5
 800038e:	f000 f937 	bl	8000600 <_fflush_r>
 8000392:	2800      	cmp	r0, #0
 8000394:	d127      	bne.n	80003e6 <__swbuf_r+0x9a>
 8000396:	68a3      	ldr	r3, [r4, #8]
 8000398:	3001      	adds	r0, #1
 800039a:	3b01      	subs	r3, #1
 800039c:	60a3      	str	r3, [r4, #8]
 800039e:	6823      	ldr	r3, [r4, #0]
 80003a0:	1c5a      	adds	r2, r3, #1
 80003a2:	6022      	str	r2, [r4, #0]
 80003a4:	701f      	strb	r7, [r3, #0]
 80003a6:	6963      	ldr	r3, [r4, #20]
 80003a8:	4283      	cmp	r3, r0
 80003aa:	d004      	beq.n	80003b6 <__swbuf_r+0x6a>
 80003ac:	89a3      	ldrh	r3, [r4, #12]
 80003ae:	07db      	lsls	r3, r3, #31
 80003b0:	d507      	bpl.n	80003c2 <__swbuf_r+0x76>
 80003b2:	2e0a      	cmp	r6, #10
 80003b4:	d105      	bne.n	80003c2 <__swbuf_r+0x76>
 80003b6:	0021      	movs	r1, r4
 80003b8:	0028      	movs	r0, r5
 80003ba:	f000 f921 	bl	8000600 <_fflush_r>
 80003be:	2800      	cmp	r0, #0
 80003c0:	d111      	bne.n	80003e6 <__swbuf_r+0x9a>
 80003c2:	0030      	movs	r0, r6
 80003c4:	bdf8      	pop	{r3, r4, r5, r6, r7, pc}
 80003c6:	4b0a      	ldr	r3, [pc, #40]	; (80003f0 <__swbuf_r+0xa4>)
 80003c8:	429c      	cmp	r4, r3
 80003ca:	d101      	bne.n	80003d0 <__swbuf_r+0x84>
 80003cc:	68ac      	ldr	r4, [r5, #8]
 80003ce:	e7cc      	b.n	800036a <__swbuf_r+0x1e>
 80003d0:	4b08      	ldr	r3, [pc, #32]	; (80003f4 <__swbuf_r+0xa8>)
 80003d2:	429c      	cmp	r4, r3
 80003d4:	d1c9      	bne.n	800036a <__swbuf_r+0x1e>
 80003d6:	68ec      	ldr	r4, [r5, #12]
 80003d8:	e7c7      	b.n	800036a <__swbuf_r+0x1e>
 80003da:	0021      	movs	r1, r4
 80003dc:	0028      	movs	r0, r5
 80003de:	f000 f80b 	bl	80003f8 <__swsetup_r>
 80003e2:	2800      	cmp	r0, #0
 80003e4:	d0c9      	beq.n	800037a <__swbuf_r+0x2e>
 80003e6:	2601      	movs	r6, #1
 80003e8:	4276      	negs	r6, r6
 80003ea:	e7ea      	b.n	80003c2 <__swbuf_r+0x76>
 80003ec:	08001260 	.word	0x08001260
 80003f0:	08001280 	.word	0x08001280
 80003f4:	08001240 	.word	0x08001240

080003f8 <__swsetup_r>:
 80003f8:	4b37      	ldr	r3, [pc, #220]	; (80004d8 <__swsetup_r+0xe0>)
 80003fa:	b570      	push	{r4, r5, r6, lr}
 80003fc:	681d      	ldr	r5, [r3, #0]
 80003fe:	0006      	movs	r6, r0
 8000400:	000c      	movs	r4, r1
 8000402:	2d00      	cmp	r5, #0
 8000404:	d005      	beq.n	8000412 <__swsetup_r+0x1a>
 8000406:	69ab      	ldr	r3, [r5, #24]
 8000408:	2b00      	cmp	r3, #0
 800040a:	d102      	bne.n	8000412 <__swsetup_r+0x1a>
 800040c:	0028      	movs	r0, r5
 800040e:	f000 f999 	bl	8000744 <__sinit>
 8000412:	4b32      	ldr	r3, [pc, #200]	; (80004dc <__swsetup_r+0xe4>)
 8000414:	429c      	cmp	r4, r3
 8000416:	d10f      	bne.n	8000438 <__swsetup_r+0x40>
 8000418:	686c      	ldr	r4, [r5, #4]
 800041a:	230c      	movs	r3, #12
 800041c:	5ee2      	ldrsh	r2, [r4, r3]
 800041e:	b293      	uxth	r3, r2
 8000420:	0711      	lsls	r1, r2, #28
 8000422:	d42d      	bmi.n	8000480 <__swsetup_r+0x88>
 8000424:	06d9      	lsls	r1, r3, #27
 8000426:	d411      	bmi.n	800044c <__swsetup_r+0x54>
 8000428:	2309      	movs	r3, #9
 800042a:	2001      	movs	r0, #1
 800042c:	6033      	str	r3, [r6, #0]
 800042e:	3337      	adds	r3, #55	; 0x37
 8000430:	4313      	orrs	r3, r2
 8000432:	81a3      	strh	r3, [r4, #12]
 8000434:	4240      	negs	r0, r0
 8000436:	bd70      	pop	{r4, r5, r6, pc}
 8000438:	4b29      	ldr	r3, [pc, #164]	; (80004e0 <__swsetup_r+0xe8>)
 800043a:	429c      	cmp	r4, r3
 800043c:	d101      	bne.n	8000442 <__swsetup_r+0x4a>
 800043e:	68ac      	ldr	r4, [r5, #8]
 8000440:	e7eb      	b.n	800041a <__swsetup_r+0x22>
 8000442:	4b28      	ldr	r3, [pc, #160]	; (80004e4 <__swsetup_r+0xec>)
 8000444:	429c      	cmp	r4, r3
 8000446:	d1e8      	bne.n	800041a <__swsetup_r+0x22>
 8000448:	68ec      	ldr	r4, [r5, #12]
 800044a:	e7e6      	b.n	800041a <__swsetup_r+0x22>
 800044c:	075b      	lsls	r3, r3, #29
 800044e:	d513      	bpl.n	8000478 <__swsetup_r+0x80>
 8000450:	6b61      	ldr	r1, [r4, #52]	; 0x34
 8000452:	2900      	cmp	r1, #0
 8000454:	d008      	beq.n	8000468 <__swsetup_r+0x70>
 8000456:	0023      	movs	r3, r4
 8000458:	3344      	adds	r3, #68	; 0x44
 800045a:	4299      	cmp	r1, r3
 800045c:	d002      	beq.n	8000464 <__swsetup_r+0x6c>
 800045e:	0030      	movs	r0, r6
 8000460:	f000 fa80 	bl	8000964 <_free_r>
 8000464:	2300      	movs	r3, #0
 8000466:	6363      	str	r3, [r4, #52]	; 0x34
 8000468:	2224      	movs	r2, #36	; 0x24
 800046a:	89a3      	ldrh	r3, [r4, #12]
 800046c:	4393      	bics	r3, r2
 800046e:	81a3      	strh	r3, [r4, #12]
 8000470:	2300      	movs	r3, #0
 8000472:	6063      	str	r3, [r4, #4]
 8000474:	6923      	ldr	r3, [r4, #16]
 8000476:	6023      	str	r3, [r4, #0]
 8000478:	2308      	movs	r3, #8
 800047a:	89a2      	ldrh	r2, [r4, #12]
 800047c:	4313      	orrs	r3, r2
 800047e:	81a3      	strh	r3, [r4, #12]
 8000480:	6923      	ldr	r3, [r4, #16]
 8000482:	2b00      	cmp	r3, #0
 8000484:	d10b      	bne.n	800049e <__swsetup_r+0xa6>
 8000486:	21a0      	movs	r1, #160	; 0xa0
 8000488:	2280      	movs	r2, #128	; 0x80
 800048a:	89a3      	ldrh	r3, [r4, #12]
 800048c:	0089      	lsls	r1, r1, #2
 800048e:	0092      	lsls	r2, r2, #2
 8000490:	400b      	ands	r3, r1
 8000492:	4293      	cmp	r3, r2
 8000494:	d003      	beq.n	800049e <__swsetup_r+0xa6>
 8000496:	0021      	movs	r1, r4
 8000498:	0030      	movs	r0, r6
 800049a:	f000 fa1f 	bl	80008dc <__smakebuf_r>
 800049e:	220c      	movs	r2, #12
 80004a0:	5ea3      	ldrsh	r3, [r4, r2]
 80004a2:	2001      	movs	r0, #1
 80004a4:	001a      	movs	r2, r3
 80004a6:	b299      	uxth	r1, r3
 80004a8:	4002      	ands	r2, r0
 80004aa:	4203      	tst	r3, r0
 80004ac:	d00f      	beq.n	80004ce <__swsetup_r+0xd6>
 80004ae:	2200      	movs	r2, #0
 80004b0:	60a2      	str	r2, [r4, #8]
 80004b2:	6962      	ldr	r2, [r4, #20]
 80004b4:	4252      	negs	r2, r2
 80004b6:	61a2      	str	r2, [r4, #24]
 80004b8:	2000      	movs	r0, #0
 80004ba:	6922      	ldr	r2, [r4, #16]
 80004bc:	4282      	cmp	r2, r0
 80004be:	d1ba      	bne.n	8000436 <__swsetup_r+0x3e>
 80004c0:	060a      	lsls	r2, r1, #24
 80004c2:	d5b8      	bpl.n	8000436 <__swsetup_r+0x3e>
 80004c4:	2240      	movs	r2, #64	; 0x40
 80004c6:	4313      	orrs	r3, r2
 80004c8:	81a3      	strh	r3, [r4, #12]
 80004ca:	3801      	subs	r0, #1
 80004cc:	e7b3      	b.n	8000436 <__swsetup_r+0x3e>
 80004ce:	0788      	lsls	r0, r1, #30
 80004d0:	d400      	bmi.n	80004d4 <__swsetup_r+0xdc>
 80004d2:	6962      	ldr	r2, [r4, #20]
 80004d4:	60a2      	str	r2, [r4, #8]
 80004d6:	e7ef      	b.n	80004b8 <__swsetup_r+0xc0>
 80004d8:	20000000 	.word	0x20000000
 80004dc:	08001260 	.word	0x08001260
 80004e0:	08001280 	.word	0x08001280
 80004e4:	08001240 	.word	0x08001240

080004e8 <__sflush_r>:
 80004e8:	b5f7      	push	{r0, r1, r2, r4, r5, r6, r7, lr}
 80004ea:	898b      	ldrh	r3, [r1, #12]
 80004ec:	0005      	movs	r5, r0
 80004ee:	000c      	movs	r4, r1
 80004f0:	071a      	lsls	r2, r3, #28
 80004f2:	d45f      	bmi.n	80005b4 <__sflush_r+0xcc>
 80004f4:	684a      	ldr	r2, [r1, #4]
 80004f6:	2a00      	cmp	r2, #0
 80004f8:	dc04      	bgt.n	8000504 <__sflush_r+0x1c>
 80004fa:	6c0a      	ldr	r2, [r1, #64]	; 0x40
 80004fc:	2a00      	cmp	r2, #0
 80004fe:	dc01      	bgt.n	8000504 <__sflush_r+0x1c>
 8000500:	2000      	movs	r0, #0
 8000502:	bdfe      	pop	{r1, r2, r3, r4, r5, r6, r7, pc}
 8000504:	6ae7      	ldr	r7, [r4, #44]	; 0x2c
 8000506:	2f00      	cmp	r7, #0
 8000508:	d0fa      	beq.n	8000500 <__sflush_r+0x18>
 800050a:	2200      	movs	r2, #0
 800050c:	2180      	movs	r1, #128	; 0x80
 800050e:	682e      	ldr	r6, [r5, #0]
 8000510:	602a      	str	r2, [r5, #0]
 8000512:	001a      	movs	r2, r3
 8000514:	0149      	lsls	r1, r1, #5
 8000516:	400a      	ands	r2, r1
 8000518:	420b      	tst	r3, r1
 800051a:	d034      	beq.n	8000586 <__sflush_r+0x9e>
 800051c:	6d60      	ldr	r0, [r4, #84]	; 0x54
 800051e:	89a3      	ldrh	r3, [r4, #12]
 8000520:	075b      	lsls	r3, r3, #29
 8000522:	d506      	bpl.n	8000532 <__sflush_r+0x4a>
 8000524:	6863      	ldr	r3, [r4, #4]
 8000526:	1ac0      	subs	r0, r0, r3
 8000528:	6b63      	ldr	r3, [r4, #52]	; 0x34
 800052a:	2b00      	cmp	r3, #0
 800052c:	d001      	beq.n	8000532 <__sflush_r+0x4a>
 800052e:	6c23      	ldr	r3, [r4, #64]	; 0x40
 8000530:	1ac0      	subs	r0, r0, r3
 8000532:	0002      	movs	r2, r0
 8000534:	6a21      	ldr	r1, [r4, #32]
 8000536:	2300      	movs	r3, #0
 8000538:	0028      	movs	r0, r5
 800053a:	6ae7      	ldr	r7, [r4, #44]	; 0x2c
 800053c:	47b8      	blx	r7
 800053e:	89a1      	ldrh	r1, [r4, #12]
 8000540:	1c43      	adds	r3, r0, #1
 8000542:	d106      	bne.n	8000552 <__sflush_r+0x6a>
 8000544:	682b      	ldr	r3, [r5, #0]
 8000546:	2b1d      	cmp	r3, #29
 8000548:	d831      	bhi.n	80005ae <__sflush_r+0xc6>
 800054a:	4a2c      	ldr	r2, [pc, #176]	; (80005fc <__sflush_r+0x114>)
 800054c:	40da      	lsrs	r2, r3
 800054e:	07d3      	lsls	r3, r2, #31
 8000550:	d52d      	bpl.n	80005ae <__sflush_r+0xc6>
 8000552:	2300      	movs	r3, #0
 8000554:	6063      	str	r3, [r4, #4]
 8000556:	6923      	ldr	r3, [r4, #16]
 8000558:	6023      	str	r3, [r4, #0]
 800055a:	04cb      	lsls	r3, r1, #19
 800055c:	d505      	bpl.n	800056a <__sflush_r+0x82>
 800055e:	1c43      	adds	r3, r0, #1
 8000560:	d102      	bne.n	8000568 <__sflush_r+0x80>
 8000562:	682b      	ldr	r3, [r5, #0]
 8000564:	2b00      	cmp	r3, #0
 8000566:	d100      	bne.n	800056a <__sflush_r+0x82>
 8000568:	6560      	str	r0, [r4, #84]	; 0x54
 800056a:	6b61      	ldr	r1, [r4, #52]	; 0x34
 800056c:	602e      	str	r6, [r5, #0]
 800056e:	2900      	cmp	r1, #0
 8000570:	d0c6      	beq.n	8000500 <__sflush_r+0x18>
 8000572:	0023      	movs	r3, r4
 8000574:	3344      	adds	r3, #68	; 0x44
 8000576:	4299      	cmp	r1, r3
 8000578:	d002      	beq.n	8000580 <__sflush_r+0x98>
 800057a:	0028      	movs	r0, r5
 800057c:	f000 f9f2 	bl	8000964 <_free_r>
 8000580:	2000      	movs	r0, #0
 8000582:	6360      	str	r0, [r4, #52]	; 0x34
 8000584:	e7bd      	b.n	8000502 <__sflush_r+0x1a>
 8000586:	2301      	movs	r3, #1
 8000588:	0028      	movs	r0, r5
 800058a:	6a21      	ldr	r1, [r4, #32]
 800058c:	47b8      	blx	r7
 800058e:	1c43      	adds	r3, r0, #1
 8000590:	d1c5      	bne.n	800051e <__sflush_r+0x36>
 8000592:	682b      	ldr	r3, [r5, #0]
 8000594:	2b00      	cmp	r3, #0
 8000596:	d0c2      	beq.n	800051e <__sflush_r+0x36>
 8000598:	2b1d      	cmp	r3, #29
 800059a:	d001      	beq.n	80005a0 <__sflush_r+0xb8>
 800059c:	2b16      	cmp	r3, #22
 800059e:	d101      	bne.n	80005a4 <__sflush_r+0xbc>
 80005a0:	602e      	str	r6, [r5, #0]
 80005a2:	e7ad      	b.n	8000500 <__sflush_r+0x18>
 80005a4:	2340      	movs	r3, #64	; 0x40
 80005a6:	89a2      	ldrh	r2, [r4, #12]
 80005a8:	4313      	orrs	r3, r2
 80005aa:	81a3      	strh	r3, [r4, #12]
 80005ac:	e7a9      	b.n	8000502 <__sflush_r+0x1a>
 80005ae:	2340      	movs	r3, #64	; 0x40
 80005b0:	430b      	orrs	r3, r1
 80005b2:	e7fa      	b.n	80005aa <__sflush_r+0xc2>
 80005b4:	690f      	ldr	r7, [r1, #16]
 80005b6:	2f00      	cmp	r7, #0
 80005b8:	d0a2      	beq.n	8000500 <__sflush_r+0x18>
 80005ba:	680a      	ldr	r2, [r1, #0]
 80005bc:	600f      	str	r7, [r1, #0]
 80005be:	1bd2      	subs	r2, r2, r7
 80005c0:	9201      	str	r2, [sp, #4]
 80005c2:	2200      	movs	r2, #0
 80005c4:	079b      	lsls	r3, r3, #30
 80005c6:	d100      	bne.n	80005ca <__sflush_r+0xe2>
 80005c8:	694a      	ldr	r2, [r1, #20]
 80005ca:	60a2      	str	r2, [r4, #8]
 80005cc:	9b01      	ldr	r3, [sp, #4]
 80005ce:	2b00      	cmp	r3, #0
 80005d0:	dc00      	bgt.n	80005d4 <__sflush_r+0xec>
 80005d2:	e795      	b.n	8000500 <__sflush_r+0x18>
 80005d4:	003a      	movs	r2, r7
 80005d6:	0028      	movs	r0, r5
 80005d8:	9b01      	ldr	r3, [sp, #4]
 80005da:	6a21      	ldr	r1, [r4, #32]
 80005dc:	6aa6      	ldr	r6, [r4, #40]	; 0x28
 80005de:	47b0      	blx	r6
 80005e0:	2800      	cmp	r0, #0
 80005e2:	dc06      	bgt.n	80005f2 <__sflush_r+0x10a>
 80005e4:	2340      	movs	r3, #64	; 0x40
 80005e6:	2001      	movs	r0, #1
 80005e8:	89a2      	ldrh	r2, [r4, #12]
 80005ea:	4240      	negs	r0, r0
 80005ec:	4313      	orrs	r3, r2
 80005ee:	81a3      	strh	r3, [r4, #12]
 80005f0:	e787      	b.n	8000502 <__sflush_r+0x1a>
 80005f2:	9b01      	ldr	r3, [sp, #4]
 80005f4:	183f      	adds	r7, r7, r0
 80005f6:	1a1b      	subs	r3, r3, r0
 80005f8:	9301      	str	r3, [sp, #4]
 80005fa:	e7e7      	b.n	80005cc <__sflush_r+0xe4>
 80005fc:	20400001 	.word	0x20400001

08000600 <_fflush_r>:
 8000600:	690b      	ldr	r3, [r1, #16]
 8000602:	b570      	push	{r4, r5, r6, lr}
 8000604:	0005      	movs	r5, r0
 8000606:	000c      	movs	r4, r1
 8000608:	2b00      	cmp	r3, #0
 800060a:	d102      	bne.n	8000612 <_fflush_r+0x12>
 800060c:	2500      	movs	r5, #0
 800060e:	0028      	movs	r0, r5
 8000610:	bd70      	pop	{r4, r5, r6, pc}
 8000612:	2800      	cmp	r0, #0
 8000614:	d004      	beq.n	8000620 <_fflush_r+0x20>
 8000616:	6983      	ldr	r3, [r0, #24]
 8000618:	2b00      	cmp	r3, #0
 800061a:	d101      	bne.n	8000620 <_fflush_r+0x20>
 800061c:	f000 f892 	bl	8000744 <__sinit>
 8000620:	4b14      	ldr	r3, [pc, #80]	; (8000674 <_fflush_r+0x74>)
 8000622:	429c      	cmp	r4, r3
 8000624:	d11b      	bne.n	800065e <_fflush_r+0x5e>
 8000626:	686c      	ldr	r4, [r5, #4]
 8000628:	220c      	movs	r2, #12
 800062a:	5ea3      	ldrsh	r3, [r4, r2]
 800062c:	2b00      	cmp	r3, #0
 800062e:	d0ed      	beq.n	800060c <_fflush_r+0xc>
 8000630:	6e62      	ldr	r2, [r4, #100]	; 0x64
 8000632:	07d2      	lsls	r2, r2, #31
 8000634:	d404      	bmi.n	8000640 <_fflush_r+0x40>
 8000636:	059b      	lsls	r3, r3, #22
 8000638:	d402      	bmi.n	8000640 <_fflush_r+0x40>
 800063a:	6da0      	ldr	r0, [r4, #88]	; 0x58
 800063c:	f000 f923 	bl	8000886 <__retarget_lock_acquire_recursive>
 8000640:	0028      	movs	r0, r5
 8000642:	0021      	movs	r1, r4
 8000644:	f7ff ff50 	bl	80004e8 <__sflush_r>
 8000648:	6e63      	ldr	r3, [r4, #100]	; 0x64
 800064a:	0005      	movs	r5, r0
 800064c:	07db      	lsls	r3, r3, #31
 800064e:	d4de      	bmi.n	800060e <_fflush_r+0xe>
 8000650:	89a3      	ldrh	r3, [r4, #12]
 8000652:	059b      	lsls	r3, r3, #22
 8000654:	d4db      	bmi.n	800060e <_fflush_r+0xe>
 8000656:	6da0      	ldr	r0, [r4, #88]	; 0x58
 8000658:	f000 f916 	bl	8000888 <__retarget_lock_release_recursive>
 800065c:	e7d7      	b.n	800060e <_fflush_r+0xe>
 800065e:	4b06      	ldr	r3, [pc, #24]	; (8000678 <_fflush_r+0x78>)
 8000660:	429c      	cmp	r4, r3
 8000662:	d101      	bne.n	8000668 <_fflush_r+0x68>
 8000664:	68ac      	ldr	r4, [r5, #8]
 8000666:	e7df      	b.n	8000628 <_fflush_r+0x28>
 8000668:	4b04      	ldr	r3, [pc, #16]	; (800067c <_fflush_r+0x7c>)
 800066a:	429c      	cmp	r4, r3
 800066c:	d1dc      	bne.n	8000628 <_fflush_r+0x28>
 800066e:	68ec      	ldr	r4, [r5, #12]
 8000670:	e7da      	b.n	8000628 <_fflush_r+0x28>
 8000672:	46c0      	nop			; (mov r8, r8)
 8000674:	08001260 	.word	0x08001260
 8000678:	08001280 	.word	0x08001280
 800067c:	08001240 	.word	0x08001240

08000680 <std>:
 8000680:	2300      	movs	r3, #0
 8000682:	b510      	push	{r4, lr}
 8000684:	0004      	movs	r4, r0
 8000686:	6003      	str	r3, [r0, #0]
 8000688:	6043      	str	r3, [r0, #4]
 800068a:	6083      	str	r3, [r0, #8]
 800068c:	8181      	strh	r1, [r0, #12]
 800068e:	6643      	str	r3, [r0, #100]	; 0x64
 8000690:	0019      	movs	r1, r3
 8000692:	81c2      	strh	r2, [r0, #14]
 8000694:	6103      	str	r3, [r0, #16]
 8000696:	6143      	str	r3, [r0, #20]
 8000698:	6183      	str	r3, [r0, #24]
 800069a:	2208      	movs	r2, #8
 800069c:	305c      	adds	r0, #92	; 0x5c
 800069e:	f7ff fdd1 	bl	8000244 <memset>
 80006a2:	4b05      	ldr	r3, [pc, #20]	; (80006b8 <std+0x38>)
 80006a4:	6224      	str	r4, [r4, #32]
 80006a6:	6263      	str	r3, [r4, #36]	; 0x24
 80006a8:	4b04      	ldr	r3, [pc, #16]	; (80006bc <std+0x3c>)
 80006aa:	62a3      	str	r3, [r4, #40]	; 0x28
 80006ac:	4b04      	ldr	r3, [pc, #16]	; (80006c0 <std+0x40>)
 80006ae:	62e3      	str	r3, [r4, #44]	; 0x2c
 80006b0:	4b04      	ldr	r3, [pc, #16]	; (80006c4 <std+0x44>)
 80006b2:	6323      	str	r3, [r4, #48]	; 0x30
 80006b4:	bd10      	pop	{r4, pc}
 80006b6:	46c0      	nop			; (mov r8, r8)
 80006b8:	08000b4d 	.word	0x08000b4d
 80006bc:	08000b75 	.word	0x08000b75
 80006c0:	08000bad 	.word	0x08000bad
 80006c4:	08000bd9 	.word	0x08000bd9

080006c8 <_cleanup_r>:
 80006c8:	b510      	push	{r4, lr}
 80006ca:	4902      	ldr	r1, [pc, #8]	; (80006d4 <_cleanup_r+0xc>)
 80006cc:	f000 f8ba 	bl	8000844 <_fwalk_reent>
 80006d0:	bd10      	pop	{r4, pc}
 80006d2:	46c0      	nop			; (mov r8, r8)
 80006d4:	08000601 	.word	0x08000601

080006d8 <__sfmoreglue>:
 80006d8:	b570      	push	{r4, r5, r6, lr}
 80006da:	2568      	movs	r5, #104	; 0x68
 80006dc:	1e4a      	subs	r2, r1, #1
 80006de:	4355      	muls	r5, r2
 80006e0:	000e      	movs	r6, r1
 80006e2:	0029      	movs	r1, r5
 80006e4:	3174      	adds	r1, #116	; 0x74
 80006e6:	f000 f9a9 	bl	8000a3c <_malloc_r>
 80006ea:	1e04      	subs	r4, r0, #0
 80006ec:	d008      	beq.n	8000700 <__sfmoreglue+0x28>
 80006ee:	2100      	movs	r1, #0
 80006f0:	002a      	movs	r2, r5
 80006f2:	6001      	str	r1, [r0, #0]
 80006f4:	6046      	str	r6, [r0, #4]
 80006f6:	300c      	adds	r0, #12
 80006f8:	60a0      	str	r0, [r4, #8]
 80006fa:	3268      	adds	r2, #104	; 0x68
 80006fc:	f7ff fda2 	bl	8000244 <memset>
 8000700:	0020      	movs	r0, r4
 8000702:	bd70      	pop	{r4, r5, r6, pc}

08000704 <__sfp_lock_acquire>:
 8000704:	b510      	push	{r4, lr}
 8000706:	4802      	ldr	r0, [pc, #8]	; (8000710 <__sfp_lock_acquire+0xc>)
 8000708:	f000 f8bd 	bl	8000886 <__retarget_lock_acquire_recursive>
 800070c:	bd10      	pop	{r4, pc}
 800070e:	46c0      	nop			; (mov r8, r8)
 8000710:	2000008d 	.word	0x2000008d

08000714 <__sfp_lock_release>:
 8000714:	b510      	push	{r4, lr}
 8000716:	4802      	ldr	r0, [pc, #8]	; (8000720 <__sfp_lock_release+0xc>)
 8000718:	f000 f8b6 	bl	8000888 <__retarget_lock_release_recursive>
 800071c:	bd10      	pop	{r4, pc}
 800071e:	46c0      	nop			; (mov r8, r8)
 8000720:	2000008d 	.word	0x2000008d

08000724 <__sinit_lock_acquire>:
 8000724:	b510      	push	{r4, lr}
 8000726:	4802      	ldr	r0, [pc, #8]	; (8000730 <__sinit_lock_acquire+0xc>)
 8000728:	f000 f8ad 	bl	8000886 <__retarget_lock_acquire_recursive>
 800072c:	bd10      	pop	{r4, pc}
 800072e:	46c0      	nop			; (mov r8, r8)
 8000730:	2000008e 	.word	0x2000008e

08000734 <__sinit_lock_release>:
 8000734:	b510      	push	{r4, lr}
 8000736:	4802      	ldr	r0, [pc, #8]	; (8000740 <__sinit_lock_release+0xc>)
 8000738:	f000 f8a6 	bl	8000888 <__retarget_lock_release_recursive>
 800073c:	bd10      	pop	{r4, pc}
 800073e:	46c0      	nop			; (mov r8, r8)
 8000740:	2000008e 	.word	0x2000008e

08000744 <__sinit>:
 8000744:	b513      	push	{r0, r1, r4, lr}
 8000746:	0004      	movs	r4, r0
 8000748:	f7ff ffec 	bl	8000724 <__sinit_lock_acquire>
 800074c:	69a3      	ldr	r3, [r4, #24]
 800074e:	2b00      	cmp	r3, #0
 8000750:	d002      	beq.n	8000758 <__sinit+0x14>
 8000752:	f7ff ffef 	bl	8000734 <__sinit_lock_release>
 8000756:	bd13      	pop	{r0, r1, r4, pc}
 8000758:	64a3      	str	r3, [r4, #72]	; 0x48
 800075a:	64e3      	str	r3, [r4, #76]	; 0x4c
 800075c:	6523      	str	r3, [r4, #80]	; 0x50
 800075e:	4b13      	ldr	r3, [pc, #76]	; (80007ac <__sinit+0x68>)
 8000760:	4a13      	ldr	r2, [pc, #76]	; (80007b0 <__sinit+0x6c>)
 8000762:	681b      	ldr	r3, [r3, #0]
 8000764:	62a2      	str	r2, [r4, #40]	; 0x28
 8000766:	9301      	str	r3, [sp, #4]
 8000768:	42a3      	cmp	r3, r4
 800076a:	d101      	bne.n	8000770 <__sinit+0x2c>
 800076c:	2301      	movs	r3, #1
 800076e:	61a3      	str	r3, [r4, #24]
 8000770:	0020      	movs	r0, r4
 8000772:	f000 f81f 	bl	80007b4 <__sfp>
 8000776:	6060      	str	r0, [r4, #4]
 8000778:	0020      	movs	r0, r4
 800077a:	f000 f81b 	bl	80007b4 <__sfp>
 800077e:	60a0      	str	r0, [r4, #8]
 8000780:	0020      	movs	r0, r4
 8000782:	f000 f817 	bl	80007b4 <__sfp>
 8000786:	2200      	movs	r2, #0
 8000788:	2104      	movs	r1, #4
 800078a:	60e0      	str	r0, [r4, #12]
 800078c:	6860      	ldr	r0, [r4, #4]
 800078e:	f7ff ff77 	bl	8000680 <std>
 8000792:	2201      	movs	r2, #1
 8000794:	2109      	movs	r1, #9
 8000796:	68a0      	ldr	r0, [r4, #8]
 8000798:	f7ff ff72 	bl	8000680 <std>
 800079c:	2202      	movs	r2, #2
 800079e:	2112      	movs	r1, #18
 80007a0:	68e0      	ldr	r0, [r4, #12]
 80007a2:	f7ff ff6d 	bl	8000680 <std>
 80007a6:	2301      	movs	r3, #1
 80007a8:	61a3      	str	r3, [r4, #24]
 80007aa:	e7d2      	b.n	8000752 <__sinit+0xe>
 80007ac:	0800123c 	.word	0x0800123c
 80007b0:	080006c9 	.word	0x080006c9

080007b4 <__sfp>:
 80007b4:	b5f8      	push	{r3, r4, r5, r6, r7, lr}
 80007b6:	0007      	movs	r7, r0
 80007b8:	f7ff ffa4 	bl	8000704 <__sfp_lock_acquire>
 80007bc:	4b1f      	ldr	r3, [pc, #124]	; (800083c <__sfp+0x88>)
 80007be:	681e      	ldr	r6, [r3, #0]
 80007c0:	69b3      	ldr	r3, [r6, #24]
 80007c2:	2b00      	cmp	r3, #0
 80007c4:	d102      	bne.n	80007cc <__sfp+0x18>
 80007c6:	0030      	movs	r0, r6
 80007c8:	f7ff ffbc 	bl	8000744 <__sinit>
 80007cc:	3648      	adds	r6, #72	; 0x48
 80007ce:	68b4      	ldr	r4, [r6, #8]
 80007d0:	6873      	ldr	r3, [r6, #4]
 80007d2:	3b01      	subs	r3, #1
 80007d4:	d504      	bpl.n	80007e0 <__sfp+0x2c>
 80007d6:	6833      	ldr	r3, [r6, #0]
 80007d8:	2b00      	cmp	r3, #0
 80007da:	d022      	beq.n	8000822 <__sfp+0x6e>
 80007dc:	6836      	ldr	r6, [r6, #0]
 80007de:	e7f6      	b.n	80007ce <__sfp+0x1a>
 80007e0:	220c      	movs	r2, #12
 80007e2:	5ea5      	ldrsh	r5, [r4, r2]
 80007e4:	2d00      	cmp	r5, #0
 80007e6:	d11a      	bne.n	800081e <__sfp+0x6a>
 80007e8:	0020      	movs	r0, r4
 80007ea:	4b15      	ldr	r3, [pc, #84]	; (8000840 <__sfp+0x8c>)
 80007ec:	3058      	adds	r0, #88	; 0x58
 80007ee:	60e3      	str	r3, [r4, #12]
 80007f0:	6665      	str	r5, [r4, #100]	; 0x64
 80007f2:	f000 f847 	bl	8000884 <__retarget_lock_init_recursive>
 80007f6:	f7ff ff8d 	bl	8000714 <__sfp_lock_release>
 80007fa:	0020      	movs	r0, r4
 80007fc:	2208      	movs	r2, #8
 80007fe:	0029      	movs	r1, r5
 8000800:	6025      	str	r5, [r4, #0]
 8000802:	60a5      	str	r5, [r4, #8]
 8000804:	6065      	str	r5, [r4, #4]
 8000806:	6125      	str	r5, [r4, #16]
 8000808:	6165      	str	r5, [r4, #20]
 800080a:	61a5      	str	r5, [r4, #24]
 800080c:	305c      	adds	r0, #92	; 0x5c
 800080e:	f7ff fd19 	bl	8000244 <memset>
 8000812:	6365      	str	r5, [r4, #52]	; 0x34
 8000814:	63a5      	str	r5, [r4, #56]	; 0x38
 8000816:	64a5      	str	r5, [r4, #72]	; 0x48
 8000818:	64e5      	str	r5, [r4, #76]	; 0x4c
 800081a:	0020      	movs	r0, r4
 800081c:	bdf8      	pop	{r3, r4, r5, r6, r7, pc}
 800081e:	3468      	adds	r4, #104	; 0x68
 8000820:	e7d7      	b.n	80007d2 <__sfp+0x1e>
 8000822:	2104      	movs	r1, #4
 8000824:	0038      	movs	r0, r7
 8000826:	f7ff ff57 	bl	80006d8 <__sfmoreglue>
 800082a:	1e04      	subs	r4, r0, #0
 800082c:	6030      	str	r0, [r6, #0]
 800082e:	d1d5      	bne.n	80007dc <__sfp+0x28>
 8000830:	f7ff ff70 	bl	8000714 <__sfp_lock_release>
 8000834:	230c      	movs	r3, #12
 8000836:	603b      	str	r3, [r7, #0]
 8000838:	e7ef      	b.n	800081a <__sfp+0x66>
 800083a:	46c0      	nop			; (mov r8, r8)
 800083c:	0800123c 	.word	0x0800123c
 8000840:	ffff0001 	.word	0xffff0001

08000844 <_fwalk_reent>:
 8000844:	b5f7      	push	{r0, r1, r2, r4, r5, r6, r7, lr}
 8000846:	0004      	movs	r4, r0
 8000848:	0006      	movs	r6, r0
 800084a:	2700      	movs	r7, #0
 800084c:	9101      	str	r1, [sp, #4]
 800084e:	3448      	adds	r4, #72	; 0x48
 8000850:	6863      	ldr	r3, [r4, #4]
 8000852:	68a5      	ldr	r5, [r4, #8]
 8000854:	9300      	str	r3, [sp, #0]
 8000856:	9b00      	ldr	r3, [sp, #0]
 8000858:	3b01      	subs	r3, #1
 800085a:	9300      	str	r3, [sp, #0]
 800085c:	d504      	bpl.n	8000868 <_fwalk_reent+0x24>
 800085e:	6824      	ldr	r4, [r4, #0]
 8000860:	2c00      	cmp	r4, #0
 8000862:	d1f5      	bne.n	8000850 <_fwalk_reent+0xc>
 8000864:	0038      	movs	r0, r7
 8000866:	bdfe      	pop	{r1, r2, r3, r4, r5, r6, r7, pc}
 8000868:	89ab      	ldrh	r3, [r5, #12]
 800086a:	2b01      	cmp	r3, #1
 800086c:	d908      	bls.n	8000880 <_fwalk_reent+0x3c>
 800086e:	220e      	movs	r2, #14
 8000870:	5eab      	ldrsh	r3, [r5, r2]
 8000872:	3301      	adds	r3, #1
 8000874:	d004      	beq.n	8000880 <_fwalk_reent+0x3c>
 8000876:	0029      	movs	r1, r5
 8000878:	0030      	movs	r0, r6
 800087a:	9b01      	ldr	r3, [sp, #4]
 800087c:	4798      	blx	r3
 800087e:	4307      	orrs	r7, r0
 8000880:	3568      	adds	r5, #104	; 0x68
 8000882:	e7e8      	b.n	8000856 <_fwalk_reent+0x12>

08000884 <__retarget_lock_init_recursive>:
 8000884:	4770      	bx	lr

08000886 <__retarget_lock_acquire_recursive>:
 8000886:	4770      	bx	lr

08000888 <__retarget_lock_release_recursive>:
 8000888:	4770      	bx	lr
	...

0800088c <__swhatbuf_r>:
 800088c:	b570      	push	{r4, r5, r6, lr}
 800088e:	000e      	movs	r6, r1
 8000890:	001d      	movs	r5, r3
 8000892:	230e      	movs	r3, #14
 8000894:	5ec9      	ldrsh	r1, [r1, r3]
 8000896:	0014      	movs	r4, r2
 8000898:	b096      	sub	sp, #88	; 0x58
 800089a:	2900      	cmp	r1, #0
 800089c:	da08      	bge.n	80008b0 <__swhatbuf_r+0x24>
 800089e:	220c      	movs	r2, #12
 80008a0:	5eb3      	ldrsh	r3, [r6, r2]
 80008a2:	2200      	movs	r2, #0
 80008a4:	602a      	str	r2, [r5, #0]
 80008a6:	061b      	lsls	r3, r3, #24
 80008a8:	d411      	bmi.n	80008ce <__swhatbuf_r+0x42>
 80008aa:	2380      	movs	r3, #128	; 0x80
 80008ac:	00db      	lsls	r3, r3, #3
 80008ae:	e00f      	b.n	80008d0 <__swhatbuf_r+0x44>
 80008b0:	466a      	mov	r2, sp
 80008b2:	f000 f9bd 	bl	8000c30 <_fstat_r>
 80008b6:	2800      	cmp	r0, #0
 80008b8:	dbf1      	blt.n	800089e <__swhatbuf_r+0x12>
 80008ba:	23f0      	movs	r3, #240	; 0xf0
 80008bc:	9901      	ldr	r1, [sp, #4]
 80008be:	021b      	lsls	r3, r3, #8
 80008c0:	4019      	ands	r1, r3
 80008c2:	4b05      	ldr	r3, [pc, #20]	; (80008d8 <__swhatbuf_r+0x4c>)
 80008c4:	18c9      	adds	r1, r1, r3
 80008c6:	424b      	negs	r3, r1
 80008c8:	4159      	adcs	r1, r3
 80008ca:	6029      	str	r1, [r5, #0]
 80008cc:	e7ed      	b.n	80008aa <__swhatbuf_r+0x1e>
 80008ce:	2340      	movs	r3, #64	; 0x40
 80008d0:	2000      	movs	r0, #0
 80008d2:	6023      	str	r3, [r4, #0]
 80008d4:	b016      	add	sp, #88	; 0x58
 80008d6:	bd70      	pop	{r4, r5, r6, pc}
 80008d8:	ffffe000 	.word	0xffffe000

080008dc <__smakebuf_r>:
 80008dc:	b5f7      	push	{r0, r1, r2, r4, r5, r6, r7, lr}
 80008de:	2602      	movs	r6, #2
 80008e0:	898b      	ldrh	r3, [r1, #12]
 80008e2:	0005      	movs	r5, r0
 80008e4:	000c      	movs	r4, r1
 80008e6:	4233      	tst	r3, r6
 80008e8:	d006      	beq.n	80008f8 <__smakebuf_r+0x1c>
 80008ea:	0023      	movs	r3, r4
 80008ec:	3347      	adds	r3, #71	; 0x47
 80008ee:	6023      	str	r3, [r4, #0]
 80008f0:	6123      	str	r3, [r4, #16]
 80008f2:	2301      	movs	r3, #1
 80008f4:	6163      	str	r3, [r4, #20]
 80008f6:	bdf7      	pop	{r0, r1, r2, r4, r5, r6, r7, pc}
 80008f8:	466a      	mov	r2, sp
 80008fa:	ab01      	add	r3, sp, #4
 80008fc:	f7ff ffc6 	bl	800088c <__swhatbuf_r>
 8000900:	9900      	ldr	r1, [sp, #0]
 8000902:	0007      	movs	r7, r0
 8000904:	0028      	movs	r0, r5
 8000906:	f000 f899 	bl	8000a3c <_malloc_r>
 800090a:	2800      	cmp	r0, #0
 800090c:	d108      	bne.n	8000920 <__smakebuf_r+0x44>
 800090e:	220c      	movs	r2, #12
 8000910:	5ea3      	ldrsh	r3, [r4, r2]
 8000912:	059a      	lsls	r2, r3, #22
 8000914:	d4ef      	bmi.n	80008f6 <__smakebuf_r+0x1a>
 8000916:	2203      	movs	r2, #3
 8000918:	4393      	bics	r3, r2
 800091a:	431e      	orrs	r6, r3
 800091c:	81a6      	strh	r6, [r4, #12]
 800091e:	e7e4      	b.n	80008ea <__smakebuf_r+0xe>
 8000920:	4b0f      	ldr	r3, [pc, #60]	; (8000960 <__smakebuf_r+0x84>)
 8000922:	62ab      	str	r3, [r5, #40]	; 0x28
 8000924:	2380      	movs	r3, #128	; 0x80
 8000926:	89a2      	ldrh	r2, [r4, #12]
 8000928:	6020      	str	r0, [r4, #0]
 800092a:	4313      	orrs	r3, r2
 800092c:	81a3      	strh	r3, [r4, #12]
 800092e:	9b00      	ldr	r3, [sp, #0]
 8000930:	6120      	str	r0, [r4, #16]
 8000932:	6163      	str	r3, [r4, #20]
 8000934:	9b01      	ldr	r3, [sp, #4]
 8000936:	2b00      	cmp	r3, #0
 8000938:	d00d      	beq.n	8000956 <__smakebuf_r+0x7a>
 800093a:	0028      	movs	r0, r5
 800093c:	230e      	movs	r3, #14
 800093e:	5ee1      	ldrsh	r1, [r4, r3]
 8000940:	f000 f988 	bl	8000c54 <_isatty_r>
 8000944:	2800      	cmp	r0, #0
 8000946:	d006      	beq.n	8000956 <__smakebuf_r+0x7a>
 8000948:	2203      	movs	r2, #3
 800094a:	89a3      	ldrh	r3, [r4, #12]
 800094c:	4393      	bics	r3, r2
 800094e:	001a      	movs	r2, r3
 8000950:	2301      	movs	r3, #1
 8000952:	4313      	orrs	r3, r2
 8000954:	81a3      	strh	r3, [r4, #12]
 8000956:	89a0      	ldrh	r0, [r4, #12]
 8000958:	4307      	orrs	r7, r0
 800095a:	81a7      	strh	r7, [r4, #12]
 800095c:	e7cb      	b.n	80008f6 <__smakebuf_r+0x1a>
 800095e:	46c0      	nop			; (mov r8, r8)
 8000960:	080006c9 	.word	0x080006c9

08000964 <_free_r>:
 8000964:	b570      	push	{r4, r5, r6, lr}
 8000966:	0005      	movs	r5, r0
 8000968:	2900      	cmp	r1, #0
 800096a:	d010      	beq.n	800098e <_free_r+0x2a>
 800096c:	1f0c      	subs	r4, r1, #4
 800096e:	6823      	ldr	r3, [r4, #0]
 8000970:	2b00      	cmp	r3, #0
 8000972:	da00      	bge.n	8000976 <_free_r+0x12>
 8000974:	18e4      	adds	r4, r4, r3
 8000976:	0028      	movs	r0, r5
 8000978:	f000 f992 	bl	8000ca0 <__malloc_lock>
 800097c:	4a1d      	ldr	r2, [pc, #116]	; (80009f4 <_free_r+0x90>)
 800097e:	6813      	ldr	r3, [r2, #0]
 8000980:	2b00      	cmp	r3, #0
 8000982:	d105      	bne.n	8000990 <_free_r+0x2c>
 8000984:	6063      	str	r3, [r4, #4]
 8000986:	6014      	str	r4, [r2, #0]
 8000988:	0028      	movs	r0, r5
 800098a:	f000 f991 	bl	8000cb0 <__malloc_unlock>
 800098e:	bd70      	pop	{r4, r5, r6, pc}
 8000990:	42a3      	cmp	r3, r4
 8000992:	d908      	bls.n	80009a6 <_free_r+0x42>
 8000994:	6821      	ldr	r1, [r4, #0]
 8000996:	1860      	adds	r0, r4, r1
 8000998:	4283      	cmp	r3, r0
 800099a:	d1f3      	bne.n	8000984 <_free_r+0x20>
 800099c:	6818      	ldr	r0, [r3, #0]
 800099e:	685b      	ldr	r3, [r3, #4]
 80009a0:	1841      	adds	r1, r0, r1
 80009a2:	6021      	str	r1, [r4, #0]
 80009a4:	e7ee      	b.n	8000984 <_free_r+0x20>
 80009a6:	001a      	movs	r2, r3
 80009a8:	685b      	ldr	r3, [r3, #4]
 80009aa:	2b00      	cmp	r3, #0
 80009ac:	d001      	beq.n	80009b2 <_free_r+0x4e>
 80009ae:	42a3      	cmp	r3, r4
 80009b0:	d9f9      	bls.n	80009a6 <_free_r+0x42>
 80009b2:	6811      	ldr	r1, [r2, #0]
 80009b4:	1850      	adds	r0, r2, r1
 80009b6:	42a0      	cmp	r0, r4
 80009b8:	d10b      	bne.n	80009d2 <_free_r+0x6e>
 80009ba:	6820      	ldr	r0, [r4, #0]
 80009bc:	1809      	adds	r1, r1, r0
 80009be:	1850      	adds	r0, r2, r1
 80009c0:	6011      	str	r1, [r2, #0]
 80009c2:	4283      	cmp	r3, r0
 80009c4:	d1e0      	bne.n	8000988 <_free_r+0x24>
 80009c6:	6818      	ldr	r0, [r3, #0]
 80009c8:	685b      	ldr	r3, [r3, #4]
 80009ca:	1841      	adds	r1, r0, r1
 80009cc:	6011      	str	r1, [r2, #0]
 80009ce:	6053      	str	r3, [r2, #4]
 80009d0:	e7da      	b.n	8000988 <_free_r+0x24>
 80009d2:	42a0      	cmp	r0, r4
 80009d4:	d902      	bls.n	80009dc <_free_r+0x78>
 80009d6:	230c      	movs	r3, #12
 80009d8:	602b      	str	r3, [r5, #0]
 80009da:	e7d5      	b.n	8000988 <_free_r+0x24>
 80009dc:	6821      	ldr	r1, [r4, #0]
 80009de:	1860      	adds	r0, r4, r1
 80009e0:	4283      	cmp	r3, r0
 80009e2:	d103      	bne.n	80009ec <_free_r+0x88>
 80009e4:	6818      	ldr	r0, [r3, #0]
 80009e6:	685b      	ldr	r3, [r3, #4]
 80009e8:	1841      	adds	r1, r0, r1
 80009ea:	6021      	str	r1, [r4, #0]
 80009ec:	6063      	str	r3, [r4, #4]
 80009ee:	6054      	str	r4, [r2, #4]
 80009f0:	e7ca      	b.n	8000988 <_free_r+0x24>
 80009f2:	46c0      	nop			; (mov r8, r8)
 80009f4:	20000090 	.word	0x20000090

080009f8 <sbrk_aligned>:
 80009f8:	b570      	push	{r4, r5, r6, lr}
 80009fa:	4e0f      	ldr	r6, [pc, #60]	; (8000a38 <sbrk_aligned+0x40>)
 80009fc:	000d      	movs	r5, r1
 80009fe:	6831      	ldr	r1, [r6, #0]
 8000a00:	0004      	movs	r4, r0
 8000a02:	2900      	cmp	r1, #0
 8000a04:	d102      	bne.n	8000a0c <sbrk_aligned+0x14>
 8000a06:	f000 f88f 	bl	8000b28 <_sbrk_r>
 8000a0a:	6030      	str	r0, [r6, #0]
 8000a0c:	0029      	movs	r1, r5
 8000a0e:	0020      	movs	r0, r4
 8000a10:	f000 f88a 	bl	8000b28 <_sbrk_r>
 8000a14:	1c43      	adds	r3, r0, #1
 8000a16:	d00a      	beq.n	8000a2e <sbrk_aligned+0x36>
 8000a18:	2303      	movs	r3, #3
 8000a1a:	1cc5      	adds	r5, r0, #3
 8000a1c:	439d      	bics	r5, r3
 8000a1e:	42a8      	cmp	r0, r5
 8000a20:	d007      	beq.n	8000a32 <sbrk_aligned+0x3a>
 8000a22:	1a29      	subs	r1, r5, r0
 8000a24:	0020      	movs	r0, r4
 8000a26:	f000 f87f 	bl	8000b28 <_sbrk_r>
 8000a2a:	1c43      	adds	r3, r0, #1
 8000a2c:	d101      	bne.n	8000a32 <sbrk_aligned+0x3a>
 8000a2e:	2501      	movs	r5, #1
 8000a30:	426d      	negs	r5, r5
 8000a32:	0028      	movs	r0, r5
 8000a34:	bd70      	pop	{r4, r5, r6, pc}
 8000a36:	46c0      	nop			; (mov r8, r8)
 8000a38:	20000094 	.word	0x20000094

08000a3c <_malloc_r>:
 8000a3c:	b5f7      	push	{r0, r1, r2, r4, r5, r6, r7, lr}
 8000a3e:	2203      	movs	r2, #3
 8000a40:	1ccb      	adds	r3, r1, #3
 8000a42:	4393      	bics	r3, r2
 8000a44:	3308      	adds	r3, #8
 8000a46:	0006      	movs	r6, r0
 8000a48:	001f      	movs	r7, r3
 8000a4a:	2b0c      	cmp	r3, #12
 8000a4c:	d232      	bcs.n	8000ab4 <_malloc_r+0x78>
 8000a4e:	270c      	movs	r7, #12
 8000a50:	42b9      	cmp	r1, r7
 8000a52:	d831      	bhi.n	8000ab8 <_malloc_r+0x7c>
 8000a54:	0030      	movs	r0, r6
 8000a56:	f000 f923 	bl	8000ca0 <__malloc_lock>
 8000a5a:	4d32      	ldr	r5, [pc, #200]	; (8000b24 <_malloc_r+0xe8>)
 8000a5c:	682b      	ldr	r3, [r5, #0]
 8000a5e:	001c      	movs	r4, r3
 8000a60:	2c00      	cmp	r4, #0
 8000a62:	d12e      	bne.n	8000ac2 <_malloc_r+0x86>
 8000a64:	0039      	movs	r1, r7
 8000a66:	0030      	movs	r0, r6
 8000a68:	f7ff ffc6 	bl	80009f8 <sbrk_aligned>
 8000a6c:	0004      	movs	r4, r0
 8000a6e:	1c43      	adds	r3, r0, #1
 8000a70:	d11e      	bne.n	8000ab0 <_malloc_r+0x74>
 8000a72:	682c      	ldr	r4, [r5, #0]
 8000a74:	0025      	movs	r5, r4
 8000a76:	2d00      	cmp	r5, #0
 8000a78:	d14a      	bne.n	8000b10 <_malloc_r+0xd4>
 8000a7a:	6823      	ldr	r3, [r4, #0]
 8000a7c:	0029      	movs	r1, r5
 8000a7e:	18e3      	adds	r3, r4, r3
 8000a80:	0030      	movs	r0, r6
 8000a82:	9301      	str	r3, [sp, #4]
 8000a84:	f000 f850 	bl	8000b28 <_sbrk_r>
 8000a88:	9b01      	ldr	r3, [sp, #4]
 8000a8a:	4283      	cmp	r3, r0
 8000a8c:	d143      	bne.n	8000b16 <_malloc_r+0xda>
 8000a8e:	6823      	ldr	r3, [r4, #0]
 8000a90:	3703      	adds	r7, #3
 8000a92:	1aff      	subs	r7, r7, r3
 8000a94:	2303      	movs	r3, #3
 8000a96:	439f      	bics	r7, r3
 8000a98:	3708      	adds	r7, #8
 8000a9a:	2f0c      	cmp	r7, #12
 8000a9c:	d200      	bcs.n	8000aa0 <_malloc_r+0x64>
 8000a9e:	270c      	movs	r7, #12
 8000aa0:	0039      	movs	r1, r7
 8000aa2:	0030      	movs	r0, r6
 8000aa4:	f7ff ffa8 	bl	80009f8 <sbrk_aligned>
 8000aa8:	1c43      	adds	r3, r0, #1
 8000aaa:	d034      	beq.n	8000b16 <_malloc_r+0xda>
 8000aac:	6823      	ldr	r3, [r4, #0]
 8000aae:	19df      	adds	r7, r3, r7
 8000ab0:	6027      	str	r7, [r4, #0]
 8000ab2:	e013      	b.n	8000adc <_malloc_r+0xa0>
 8000ab4:	2b00      	cmp	r3, #0
 8000ab6:	dacb      	bge.n	8000a50 <_malloc_r+0x14>
 8000ab8:	230c      	movs	r3, #12
 8000aba:	2500      	movs	r5, #0
 8000abc:	6033      	str	r3, [r6, #0]
 8000abe:	0028      	movs	r0, r5
 8000ac0:	bdfe      	pop	{r1, r2, r3, r4, r5, r6, r7, pc}
 8000ac2:	6822      	ldr	r2, [r4, #0]
 8000ac4:	1bd1      	subs	r1, r2, r7
 8000ac6:	d420      	bmi.n	8000b0a <_malloc_r+0xce>
 8000ac8:	290b      	cmp	r1, #11
 8000aca:	d917      	bls.n	8000afc <_malloc_r+0xc0>
 8000acc:	19e2      	adds	r2, r4, r7
 8000ace:	6027      	str	r7, [r4, #0]
 8000ad0:	42a3      	cmp	r3, r4
 8000ad2:	d111      	bne.n	8000af8 <_malloc_r+0xbc>
 8000ad4:	602a      	str	r2, [r5, #0]
 8000ad6:	6863      	ldr	r3, [r4, #4]
 8000ad8:	6011      	str	r1, [r2, #0]
 8000ada:	6053      	str	r3, [r2, #4]
 8000adc:	0030      	movs	r0, r6
 8000ade:	0025      	movs	r5, r4
 8000ae0:	f000 f8e6 	bl	8000cb0 <__malloc_unlock>
 8000ae4:	2207      	movs	r2, #7
 8000ae6:	350b      	adds	r5, #11
 8000ae8:	1d23      	adds	r3, r4, #4
 8000aea:	4395      	bics	r5, r2
 8000aec:	1aea      	subs	r2, r5, r3
 8000aee:	429d      	cmp	r5, r3
 8000af0:	d0e5      	beq.n	8000abe <_malloc_r+0x82>
 8000af2:	1b5b      	subs	r3, r3, r5
 8000af4:	50a3      	str	r3, [r4, r2]
 8000af6:	e7e2      	b.n	8000abe <_malloc_r+0x82>
 8000af8:	605a      	str	r2, [r3, #4]
 8000afa:	e7ec      	b.n	8000ad6 <_malloc_r+0x9a>
 8000afc:	6862      	ldr	r2, [r4, #4]
 8000afe:	42a3      	cmp	r3, r4
 8000b00:	d101      	bne.n	8000b06 <_malloc_r+0xca>
 8000b02:	602a      	str	r2, [r5, #0]
 8000b04:	e7ea      	b.n	8000adc <_malloc_r+0xa0>
 8000b06:	605a      	str	r2, [r3, #4]
 8000b08:	e7e8      	b.n	8000adc <_malloc_r+0xa0>
 8000b0a:	0023      	movs	r3, r4
 8000b0c:	6864      	ldr	r4, [r4, #4]
 8000b0e:	e7a7      	b.n	8000a60 <_malloc_r+0x24>
 8000b10:	002c      	movs	r4, r5
 8000b12:	686d      	ldr	r5, [r5, #4]
 8000b14:	e7af      	b.n	8000a76 <_malloc_r+0x3a>
 8000b16:	230c      	movs	r3, #12
 8000b18:	0030      	movs	r0, r6
 8000b1a:	6033      	str	r3, [r6, #0]
 8000b1c:	f000 f8c8 	bl	8000cb0 <__malloc_unlock>
 8000b20:	e7cd      	b.n	8000abe <_malloc_r+0x82>
 8000b22:	46c0      	nop			; (mov r8, r8)
 8000b24:	20000090 	.word	0x20000090

08000b28 <_sbrk_r>:
 8000b28:	2300      	movs	r3, #0
 8000b2a:	b570      	push	{r4, r5, r6, lr}
 8000b2c:	4d06      	ldr	r5, [pc, #24]	; (8000b48 <_sbrk_r+0x20>)
 8000b2e:	0004      	movs	r4, r0
 8000b30:	0008      	movs	r0, r1
 8000b32:	602b      	str	r3, [r5, #0]
 8000b34:	f7ff fafc 	bl	8000130 <_sbrk>
 8000b38:	1c43      	adds	r3, r0, #1
 8000b3a:	d103      	bne.n	8000b44 <_sbrk_r+0x1c>
 8000b3c:	682b      	ldr	r3, [r5, #0]
 8000b3e:	2b00      	cmp	r3, #0
 8000b40:	d000      	beq.n	8000b44 <_sbrk_r+0x1c>
 8000b42:	6023      	str	r3, [r4, #0]
 8000b44:	bd70      	pop	{r4, r5, r6, pc}
 8000b46:	46c0      	nop			; (mov r8, r8)
 8000b48:	20000098 	.word	0x20000098

08000b4c <__sread>:
 8000b4c:	b570      	push	{r4, r5, r6, lr}
 8000b4e:	000c      	movs	r4, r1
 8000b50:	250e      	movs	r5, #14
 8000b52:	5f49      	ldrsh	r1, [r1, r5]
 8000b54:	f000 f8b4 	bl	8000cc0 <_read_r>
 8000b58:	2800      	cmp	r0, #0
 8000b5a:	db03      	blt.n	8000b64 <__sread+0x18>
 8000b5c:	6d63      	ldr	r3, [r4, #84]	; 0x54
 8000b5e:	181b      	adds	r3, r3, r0
 8000b60:	6563      	str	r3, [r4, #84]	; 0x54
 8000b62:	bd70      	pop	{r4, r5, r6, pc}
 8000b64:	89a3      	ldrh	r3, [r4, #12]
 8000b66:	4a02      	ldr	r2, [pc, #8]	; (8000b70 <__sread+0x24>)
 8000b68:	4013      	ands	r3, r2
 8000b6a:	81a3      	strh	r3, [r4, #12]
 8000b6c:	e7f9      	b.n	8000b62 <__sread+0x16>
 8000b6e:	46c0      	nop			; (mov r8, r8)
 8000b70:	ffffefff 	.word	0xffffefff

08000b74 <__swrite>:
 8000b74:	b5f8      	push	{r3, r4, r5, r6, r7, lr}
 8000b76:	001f      	movs	r7, r3
 8000b78:	898b      	ldrh	r3, [r1, #12]
 8000b7a:	0005      	movs	r5, r0
 8000b7c:	000c      	movs	r4, r1
 8000b7e:	0016      	movs	r6, r2
 8000b80:	05db      	lsls	r3, r3, #23
 8000b82:	d505      	bpl.n	8000b90 <__swrite+0x1c>
 8000b84:	230e      	movs	r3, #14
 8000b86:	5ec9      	ldrsh	r1, [r1, r3]
 8000b88:	2200      	movs	r2, #0
 8000b8a:	2302      	movs	r3, #2
 8000b8c:	f000 f874 	bl	8000c78 <_lseek_r>
 8000b90:	89a3      	ldrh	r3, [r4, #12]
 8000b92:	4a05      	ldr	r2, [pc, #20]	; (8000ba8 <__swrite+0x34>)
 8000b94:	0028      	movs	r0, r5
 8000b96:	4013      	ands	r3, r2
 8000b98:	81a3      	strh	r3, [r4, #12]
 8000b9a:	0032      	movs	r2, r6
 8000b9c:	230e      	movs	r3, #14
 8000b9e:	5ee1      	ldrsh	r1, [r4, r3]
 8000ba0:	003b      	movs	r3, r7
 8000ba2:	f000 f81f 	bl	8000be4 <_write_r>
 8000ba6:	bdf8      	pop	{r3, r4, r5, r6, r7, pc}
 8000ba8:	ffffefff 	.word	0xffffefff

08000bac <__sseek>:
 8000bac:	b570      	push	{r4, r5, r6, lr}
 8000bae:	000c      	movs	r4, r1
 8000bb0:	250e      	movs	r5, #14
 8000bb2:	5f49      	ldrsh	r1, [r1, r5]
 8000bb4:	f000 f860 	bl	8000c78 <_lseek_r>
 8000bb8:	89a3      	ldrh	r3, [r4, #12]
 8000bba:	1c42      	adds	r2, r0, #1
 8000bbc:	d103      	bne.n	8000bc6 <__sseek+0x1a>
 8000bbe:	4a05      	ldr	r2, [pc, #20]	; (8000bd4 <__sseek+0x28>)
 8000bc0:	4013      	ands	r3, r2
 8000bc2:	81a3      	strh	r3, [r4, #12]
 8000bc4:	bd70      	pop	{r4, r5, r6, pc}
 8000bc6:	2280      	movs	r2, #128	; 0x80
 8000bc8:	0152      	lsls	r2, r2, #5
 8000bca:	4313      	orrs	r3, r2
 8000bcc:	81a3      	strh	r3, [r4, #12]
 8000bce:	6560      	str	r0, [r4, #84]	; 0x54
 8000bd0:	e7f8      	b.n	8000bc4 <__sseek+0x18>
 8000bd2:	46c0      	nop			; (mov r8, r8)
 8000bd4:	ffffefff 	.word	0xffffefff

08000bd8 <__sclose>:
 8000bd8:	b510      	push	{r4, lr}
 8000bda:	230e      	movs	r3, #14
 8000bdc:	5ec9      	ldrsh	r1, [r1, r3]
 8000bde:	f000 f815 	bl	8000c0c <_close_r>
 8000be2:	bd10      	pop	{r4, pc}

08000be4 <_write_r>:
 8000be4:	b570      	push	{r4, r5, r6, lr}
 8000be6:	0004      	movs	r4, r0
 8000be8:	0008      	movs	r0, r1
 8000bea:	0011      	movs	r1, r2
 8000bec:	001a      	movs	r2, r3
 8000bee:	2300      	movs	r3, #0
 8000bf0:	4d05      	ldr	r5, [pc, #20]	; (8000c08 <_write_r+0x24>)
 8000bf2:	602b      	str	r3, [r5, #0]
 8000bf4:	f000 f91f 	bl	8000e36 <_write>
 8000bf8:	1c43      	adds	r3, r0, #1
 8000bfa:	d103      	bne.n	8000c04 <_write_r+0x20>
 8000bfc:	682b      	ldr	r3, [r5, #0]
 8000bfe:	2b00      	cmp	r3, #0
 8000c00:	d000      	beq.n	8000c04 <_write_r+0x20>
 8000c02:	6023      	str	r3, [r4, #0]
 8000c04:	bd70      	pop	{r4, r5, r6, pc}
 8000c06:	46c0      	nop			; (mov r8, r8)
 8000c08:	20000098 	.word	0x20000098

08000c0c <_close_r>:
 8000c0c:	2300      	movs	r3, #0
 8000c0e:	b570      	push	{r4, r5, r6, lr}
 8000c10:	4d06      	ldr	r5, [pc, #24]	; (8000c2c <_close_r+0x20>)
 8000c12:	0004      	movs	r4, r0
 8000c14:	0008      	movs	r0, r1
 8000c16:	602b      	str	r3, [r5, #0]
 8000c18:	f000 f938 	bl	8000e8c <_close>
 8000c1c:	1c43      	adds	r3, r0, #1
 8000c1e:	d103      	bne.n	8000c28 <_close_r+0x1c>
 8000c20:	682b      	ldr	r3, [r5, #0]
 8000c22:	2b00      	cmp	r3, #0
 8000c24:	d000      	beq.n	8000c28 <_close_r+0x1c>
 8000c26:	6023      	str	r3, [r4, #0]
 8000c28:	bd70      	pop	{r4, r5, r6, pc}
 8000c2a:	46c0      	nop			; (mov r8, r8)
 8000c2c:	20000098 	.word	0x20000098

08000c30 <_fstat_r>:
 8000c30:	2300      	movs	r3, #0
 8000c32:	b570      	push	{r4, r5, r6, lr}
 8000c34:	4d06      	ldr	r5, [pc, #24]	; (8000c50 <_fstat_r+0x20>)
 8000c36:	0004      	movs	r4, r0
 8000c38:	0008      	movs	r0, r1
 8000c3a:	0011      	movs	r1, r2
 8000c3c:	602b      	str	r3, [r5, #0]
 8000c3e:	f000 f96d 	bl	8000f1c <_fstat>
 8000c42:	1c43      	adds	r3, r0, #1
 8000c44:	d103      	bne.n	8000c4e <_fstat_r+0x1e>
 8000c46:	682b      	ldr	r3, [r5, #0]
 8000c48:	2b00      	cmp	r3, #0
 8000c4a:	d000      	beq.n	8000c4e <_fstat_r+0x1e>
 8000c4c:	6023      	str	r3, [r4, #0]
 8000c4e:	bd70      	pop	{r4, r5, r6, pc}
 8000c50:	20000098 	.word	0x20000098

08000c54 <_isatty_r>:
 8000c54:	2300      	movs	r3, #0
 8000c56:	b570      	push	{r4, r5, r6, lr}
 8000c58:	4d06      	ldr	r5, [pc, #24]	; (8000c74 <_isatty_r+0x20>)
 8000c5a:	0004      	movs	r4, r0
 8000c5c:	0008      	movs	r0, r1
 8000c5e:	602b      	str	r3, [r5, #0]
 8000c60:	f000 fabc 	bl	80011dc <_isatty>
 8000c64:	1c43      	adds	r3, r0, #1
 8000c66:	d103      	bne.n	8000c70 <_isatty_r+0x1c>
 8000c68:	682b      	ldr	r3, [r5, #0]
 8000c6a:	2b00      	cmp	r3, #0
 8000c6c:	d000      	beq.n	8000c70 <_isatty_r+0x1c>
 8000c6e:	6023      	str	r3, [r4, #0]
 8000c70:	bd70      	pop	{r4, r5, r6, pc}
 8000c72:	46c0      	nop			; (mov r8, r8)
 8000c74:	20000098 	.word	0x20000098

08000c78 <_lseek_r>:
 8000c78:	b570      	push	{r4, r5, r6, lr}
 8000c7a:	0004      	movs	r4, r0
 8000c7c:	0008      	movs	r0, r1
 8000c7e:	0011      	movs	r1, r2
 8000c80:	001a      	movs	r2, r3
 8000c82:	2300      	movs	r3, #0
 8000c84:	4d05      	ldr	r5, [pc, #20]	; (8000c9c <_lseek_r+0x24>)
 8000c86:	602b      	str	r3, [r5, #0]
 8000c88:	f000 f8c1 	bl	8000e0e <_lseek>
 8000c8c:	1c43      	adds	r3, r0, #1
 8000c8e:	d103      	bne.n	8000c98 <_lseek_r+0x20>
 8000c90:	682b      	ldr	r3, [r5, #0]
 8000c92:	2b00      	cmp	r3, #0
 8000c94:	d000      	beq.n	8000c98 <_lseek_r+0x20>
 8000c96:	6023      	str	r3, [r4, #0]
 8000c98:	bd70      	pop	{r4, r5, r6, pc}
 8000c9a:	46c0      	nop			; (mov r8, r8)
 8000c9c:	20000098 	.word	0x20000098

08000ca0 <__malloc_lock>:
 8000ca0:	b510      	push	{r4, lr}
 8000ca2:	4802      	ldr	r0, [pc, #8]	; (8000cac <__malloc_lock+0xc>)
 8000ca4:	f7ff fdef 	bl	8000886 <__retarget_lock_acquire_recursive>
 8000ca8:	bd10      	pop	{r4, pc}
 8000caa:	46c0      	nop			; (mov r8, r8)
 8000cac:	2000008c 	.word	0x2000008c

08000cb0 <__malloc_unlock>:
 8000cb0:	b510      	push	{r4, lr}
 8000cb2:	4802      	ldr	r0, [pc, #8]	; (8000cbc <__malloc_unlock+0xc>)
 8000cb4:	f7ff fde8 	bl	8000888 <__retarget_lock_release_recursive>
 8000cb8:	bd10      	pop	{r4, pc}
 8000cba:	46c0      	nop			; (mov r8, r8)
 8000cbc:	2000008c 	.word	0x2000008c

08000cc0 <_read_r>:
 8000cc0:	b570      	push	{r4, r5, r6, lr}
 8000cc2:	0004      	movs	r4, r0
 8000cc4:	0008      	movs	r0, r1
 8000cc6:	0011      	movs	r1, r2
 8000cc8:	001a      	movs	r2, r3
 8000cca:	2300      	movs	r3, #0
 8000ccc:	4d05      	ldr	r5, [pc, #20]	; (8000ce4 <_read_r+0x24>)
 8000cce:	602b      	str	r3, [r5, #0]
 8000cd0:	f000 f848 	bl	8000d64 <_read>
 8000cd4:	1c43      	adds	r3, r0, #1
 8000cd6:	d103      	bne.n	8000ce0 <_read_r+0x20>
 8000cd8:	682b      	ldr	r3, [r5, #0]
 8000cda:	2b00      	cmp	r3, #0
 8000cdc:	d000      	beq.n	8000ce0 <_read_r+0x20>
 8000cde:	6023      	str	r3, [r4, #0]
 8000ce0:	bd70      	pop	{r4, r5, r6, pc}
 8000ce2:	46c0      	nop			; (mov r8, r8)
 8000ce4:	20000098 	.word	0x20000098

08000ce8 <findslot>:
 8000ce8:	4b0a      	ldr	r3, [pc, #40]	; (8000d14 <findslot+0x2c>)
 8000cea:	b510      	push	{r4, lr}
 8000cec:	0004      	movs	r4, r0
 8000cee:	6818      	ldr	r0, [r3, #0]
 8000cf0:	2800      	cmp	r0, #0
 8000cf2:	d004      	beq.n	8000cfe <findslot+0x16>
 8000cf4:	6983      	ldr	r3, [r0, #24]
 8000cf6:	2b00      	cmp	r3, #0
 8000cf8:	d101      	bne.n	8000cfe <findslot+0x16>
 8000cfa:	f7ff fd23 	bl	8000744 <__sinit>
 8000cfe:	2000      	movs	r0, #0
 8000d00:	2c13      	cmp	r4, #19
 8000d02:	d805      	bhi.n	8000d10 <findslot+0x28>
 8000d04:	4b04      	ldr	r3, [pc, #16]	; (8000d18 <findslot+0x30>)
 8000d06:	00e4      	lsls	r4, r4, #3
 8000d08:	58e2      	ldr	r2, [r4, r3]
 8000d0a:	3201      	adds	r2, #1
 8000d0c:	d000      	beq.n	8000d10 <findslot+0x28>
 8000d0e:	18e0      	adds	r0, r4, r3
 8000d10:	bd10      	pop	{r4, pc}
 8000d12:	46c0      	nop			; (mov r8, r8)
 8000d14:	20000000 	.word	0x20000000
 8000d18:	200000a8 	.word	0x200000a8

08000d1c <error>:
 8000d1c:	b5f8      	push	{r3, r4, r5, r6, r7, lr}
 8000d1e:	0004      	movs	r4, r0
 8000d20:	f7ff fa66 	bl	80001f0 <__errno>
 8000d24:	2613      	movs	r6, #19
 8000d26:	0005      	movs	r5, r0
 8000d28:	2700      	movs	r7, #0
 8000d2a:	1c30      	adds	r0, r6, #0
 8000d2c:	1c39      	adds	r1, r7, #0
 8000d2e:	beab      	bkpt	0x00ab
 8000d30:	1c06      	adds	r6, r0, #0
 8000d32:	602e      	str	r6, [r5, #0]
 8000d34:	0020      	movs	r0, r4
 8000d36:	bdf8      	pop	{r3, r4, r5, r6, r7, pc}

08000d38 <checkerror>:
 8000d38:	b510      	push	{r4, lr}
 8000d3a:	1c43      	adds	r3, r0, #1
 8000d3c:	d101      	bne.n	8000d42 <checkerror+0xa>
 8000d3e:	f7ff ffed 	bl	8000d1c <error>
 8000d42:	bd10      	pop	{r4, pc}

08000d44 <_swiread>:
 8000d44:	b530      	push	{r4, r5, lr}
 8000d46:	b085      	sub	sp, #20
 8000d48:	ad01      	add	r5, sp, #4
 8000d4a:	9001      	str	r0, [sp, #4]
 8000d4c:	9102      	str	r1, [sp, #8]
 8000d4e:	9203      	str	r2, [sp, #12]
 8000d50:	2406      	movs	r4, #6
 8000d52:	1c20      	adds	r0, r4, #0
 8000d54:	1c29      	adds	r1, r5, #0
 8000d56:	beab      	bkpt	0x00ab
 8000d58:	1c04      	adds	r4, r0, #0
 8000d5a:	0020      	movs	r0, r4
 8000d5c:	f7ff ffec 	bl	8000d38 <checkerror>
 8000d60:	b005      	add	sp, #20
 8000d62:	bd30      	pop	{r4, r5, pc}

08000d64 <_read>:
 8000d64:	b570      	push	{r4, r5, r6, lr}
 8000d66:	000e      	movs	r6, r1
 8000d68:	0015      	movs	r5, r2
 8000d6a:	f7ff ffbd 	bl	8000ce8 <findslot>
 8000d6e:	1e04      	subs	r4, r0, #0
 8000d70:	d106      	bne.n	8000d80 <_read+0x1c>
 8000d72:	f7ff fa3d 	bl	80001f0 <__errno>
 8000d76:	2309      	movs	r3, #9
 8000d78:	6003      	str	r3, [r0, #0]
 8000d7a:	2001      	movs	r0, #1
 8000d7c:	4240      	negs	r0, r0
 8000d7e:	bd70      	pop	{r4, r5, r6, pc}
 8000d80:	002a      	movs	r2, r5
 8000d82:	0031      	movs	r1, r6
 8000d84:	6800      	ldr	r0, [r0, #0]
 8000d86:	f7ff ffdd 	bl	8000d44 <_swiread>
 8000d8a:	1c43      	adds	r3, r0, #1
 8000d8c:	d0f7      	beq.n	8000d7e <_read+0x1a>
 8000d8e:	6863      	ldr	r3, [r4, #4]
 8000d90:	1a28      	subs	r0, r5, r0
 8000d92:	181b      	adds	r3, r3, r0
 8000d94:	6063      	str	r3, [r4, #4]
 8000d96:	e7f2      	b.n	8000d7e <_read+0x1a>

08000d98 <_swilseek>:
 8000d98:	b5f7      	push	{r0, r1, r2, r4, r5, r6, r7, lr}
 8000d9a:	000c      	movs	r4, r1
 8000d9c:	0016      	movs	r6, r2
 8000d9e:	f7ff ffa3 	bl	8000ce8 <findslot>
 8000da2:	1e05      	subs	r5, r0, #0
 8000da4:	d107      	bne.n	8000db6 <_swilseek+0x1e>
 8000da6:	f7ff fa23 	bl	80001f0 <__errno>
 8000daa:	2309      	movs	r3, #9
 8000dac:	6003      	str	r3, [r0, #0]
 8000dae:	2401      	movs	r4, #1
 8000db0:	4264      	negs	r4, r4
 8000db2:	0020      	movs	r0, r4
 8000db4:	bdfe      	pop	{r1, r2, r3, r4, r5, r6, r7, pc}
 8000db6:	2e02      	cmp	r6, #2
 8000db8:	d903      	bls.n	8000dc2 <_swilseek+0x2a>
 8000dba:	f7ff fa19 	bl	80001f0 <__errno>
 8000dbe:	2316      	movs	r3, #22
 8000dc0:	e7f4      	b.n	8000dac <_swilseek+0x14>
 8000dc2:	2e01      	cmp	r6, #1
 8000dc4:	d112      	bne.n	8000dec <_swilseek+0x54>
 8000dc6:	6843      	ldr	r3, [r0, #4]
 8000dc8:	18e4      	adds	r4, r4, r3
 8000dca:	d4f6      	bmi.n	8000dba <_swilseek+0x22>
 8000dcc:	466f      	mov	r7, sp
 8000dce:	682b      	ldr	r3, [r5, #0]
 8000dd0:	260a      	movs	r6, #10
 8000dd2:	9300      	str	r3, [sp, #0]
 8000dd4:	607c      	str	r4, [r7, #4]
 8000dd6:	1c30      	adds	r0, r6, #0
 8000dd8:	1c39      	adds	r1, r7, #0
 8000dda:	beab      	bkpt	0x00ab
 8000ddc:	1c06      	adds	r6, r0, #0
 8000dde:	0030      	movs	r0, r6
 8000de0:	f7ff ffaa 	bl	8000d38 <checkerror>
 8000de4:	2800      	cmp	r0, #0
 8000de6:	dbe2      	blt.n	8000dae <_swilseek+0x16>
 8000de8:	606c      	str	r4, [r5, #4]
 8000dea:	e7e2      	b.n	8000db2 <_swilseek+0x1a>
 8000dec:	2e02      	cmp	r6, #2
 8000dee:	d1ed      	bne.n	8000dcc <_swilseek+0x34>
 8000df0:	6803      	ldr	r3, [r0, #0]
 8000df2:	466f      	mov	r7, sp
 8000df4:	9300      	str	r3, [sp, #0]
 8000df6:	360a      	adds	r6, #10
 8000df8:	1c30      	adds	r0, r6, #0
 8000dfa:	1c39      	adds	r1, r7, #0
 8000dfc:	beab      	bkpt	0x00ab
 8000dfe:	1c06      	adds	r6, r0, #0
 8000e00:	0030      	movs	r0, r6
 8000e02:	f7ff ff99 	bl	8000d38 <checkerror>
 8000e06:	1824      	adds	r4, r4, r0
 8000e08:	1c43      	adds	r3, r0, #1
 8000e0a:	d1df      	bne.n	8000dcc <_swilseek+0x34>
 8000e0c:	e7cf      	b.n	8000dae <_swilseek+0x16>

08000e0e <_lseek>:
 8000e0e:	b510      	push	{r4, lr}
 8000e10:	f7ff ffc2 	bl	8000d98 <_swilseek>
 8000e14:	bd10      	pop	{r4, pc}

08000e16 <_swiwrite>:
 8000e16:	b530      	push	{r4, r5, lr}
 8000e18:	b085      	sub	sp, #20
 8000e1a:	ad01      	add	r5, sp, #4
 8000e1c:	9001      	str	r0, [sp, #4]
 8000e1e:	9102      	str	r1, [sp, #8]
 8000e20:	9203      	str	r2, [sp, #12]
 8000e22:	2405      	movs	r4, #5
 8000e24:	1c20      	adds	r0, r4, #0
 8000e26:	1c29      	adds	r1, r5, #0
 8000e28:	beab      	bkpt	0x00ab
 8000e2a:	1c04      	adds	r4, r0, #0
 8000e2c:	0020      	movs	r0, r4
 8000e2e:	f7ff ff83 	bl	8000d38 <checkerror>
 8000e32:	b005      	add	sp, #20
 8000e34:	bd30      	pop	{r4, r5, pc}

08000e36 <_write>:
 8000e36:	b570      	push	{r4, r5, r6, lr}
 8000e38:	000e      	movs	r6, r1
 8000e3a:	0015      	movs	r5, r2
 8000e3c:	f7ff ff54 	bl	8000ce8 <findslot>
 8000e40:	1e04      	subs	r4, r0, #0
 8000e42:	d106      	bne.n	8000e52 <_write+0x1c>
 8000e44:	f7ff f9d4 	bl	80001f0 <__errno>
 8000e48:	2309      	movs	r3, #9
 8000e4a:	6003      	str	r3, [r0, #0]
 8000e4c:	2001      	movs	r0, #1
 8000e4e:	4240      	negs	r0, r0
 8000e50:	e00f      	b.n	8000e72 <_write+0x3c>
 8000e52:	002a      	movs	r2, r5
 8000e54:	0031      	movs	r1, r6
 8000e56:	6800      	ldr	r0, [r0, #0]
 8000e58:	f7ff ffdd 	bl	8000e16 <_swiwrite>
 8000e5c:	1e03      	subs	r3, r0, #0
 8000e5e:	dbf5      	blt.n	8000e4c <_write+0x16>
 8000e60:	6862      	ldr	r2, [r4, #4]
 8000e62:	1a28      	subs	r0, r5, r0
 8000e64:	1812      	adds	r2, r2, r0
 8000e66:	6062      	str	r2, [r4, #4]
 8000e68:	42ab      	cmp	r3, r5
 8000e6a:	d102      	bne.n	8000e72 <_write+0x3c>
 8000e6c:	2000      	movs	r0, #0
 8000e6e:	f7ff ff55 	bl	8000d1c <error>
 8000e72:	bd70      	pop	{r4, r5, r6, pc}

08000e74 <_swiclose>:
 8000e74:	b537      	push	{r0, r1, r2, r4, r5, lr}
 8000e76:	2402      	movs	r4, #2
 8000e78:	9001      	str	r0, [sp, #4]
 8000e7a:	ad01      	add	r5, sp, #4
 8000e7c:	1c20      	adds	r0, r4, #0
 8000e7e:	1c29      	adds	r1, r5, #0
 8000e80:	beab      	bkpt	0x00ab
 8000e82:	1c04      	adds	r4, r0, #0
 8000e84:	0020      	movs	r0, r4
 8000e86:	f7ff ff57 	bl	8000d38 <checkerror>
 8000e8a:	bd3e      	pop	{r1, r2, r3, r4, r5, pc}

08000e8c <_close>:
 8000e8c:	b570      	push	{r4, r5, r6, lr}
 8000e8e:	0005      	movs	r5, r0
 8000e90:	f7ff ff2a 	bl	8000ce8 <findslot>
 8000e94:	1e04      	subs	r4, r0, #0
 8000e96:	d106      	bne.n	8000ea6 <_close+0x1a>
 8000e98:	f7ff f9aa 	bl	80001f0 <__errno>
 8000e9c:	2309      	movs	r3, #9
 8000e9e:	6003      	str	r3, [r0, #0]
 8000ea0:	2001      	movs	r0, #1
 8000ea2:	4240      	negs	r0, r0
 8000ea4:	bd70      	pop	{r4, r5, r6, pc}
 8000ea6:	3d01      	subs	r5, #1
 8000ea8:	2d01      	cmp	r5, #1
 8000eaa:	d809      	bhi.n	8000ec0 <_close+0x34>
 8000eac:	4b09      	ldr	r3, [pc, #36]	; (8000ed4 <_close+0x48>)
 8000eae:	689a      	ldr	r2, [r3, #8]
 8000eb0:	691b      	ldr	r3, [r3, #16]
 8000eb2:	429a      	cmp	r2, r3
 8000eb4:	d104      	bne.n	8000ec0 <_close+0x34>
 8000eb6:	2301      	movs	r3, #1
 8000eb8:	425b      	negs	r3, r3
 8000eba:	6003      	str	r3, [r0, #0]
 8000ebc:	2000      	movs	r0, #0
 8000ebe:	e7f1      	b.n	8000ea4 <_close+0x18>
 8000ec0:	6820      	ldr	r0, [r4, #0]
 8000ec2:	f7ff ffd7 	bl	8000e74 <_swiclose>
 8000ec6:	2800      	cmp	r0, #0
 8000ec8:	d1ec      	bne.n	8000ea4 <_close+0x18>
 8000eca:	2301      	movs	r3, #1
 8000ecc:	425b      	negs	r3, r3
 8000ece:	6023      	str	r3, [r4, #0]
 8000ed0:	e7e8      	b.n	8000ea4 <_close+0x18>
 8000ed2:	46c0      	nop			; (mov r8, r8)
 8000ed4:	200000a8 	.word	0x200000a8

08000ed8 <_swistat>:
 8000ed8:	b570      	push	{r4, r5, r6, lr}
 8000eda:	000c      	movs	r4, r1
 8000edc:	f7ff ff04 	bl	8000ce8 <findslot>
 8000ee0:	1e05      	subs	r5, r0, #0
 8000ee2:	d106      	bne.n	8000ef2 <_swistat+0x1a>
 8000ee4:	f7ff f984 	bl	80001f0 <__errno>
 8000ee8:	2309      	movs	r3, #9
 8000eea:	6003      	str	r3, [r0, #0]
 8000eec:	2001      	movs	r0, #1
 8000eee:	4240      	negs	r0, r0
 8000ef0:	bd70      	pop	{r4, r5, r6, pc}
 8000ef2:	2380      	movs	r3, #128	; 0x80
 8000ef4:	6862      	ldr	r2, [r4, #4]
 8000ef6:	019b      	lsls	r3, r3, #6
 8000ef8:	4313      	orrs	r3, r2
 8000efa:	6063      	str	r3, [r4, #4]
 8000efc:	2380      	movs	r3, #128	; 0x80
 8000efe:	00db      	lsls	r3, r3, #3
 8000f00:	260c      	movs	r6, #12
 8000f02:	64a3      	str	r3, [r4, #72]	; 0x48
 8000f04:	1c30      	adds	r0, r6, #0
 8000f06:	1c29      	adds	r1, r5, #0
 8000f08:	beab      	bkpt	0x00ab
 8000f0a:	1c05      	adds	r5, r0, #0
 8000f0c:	0028      	movs	r0, r5
 8000f0e:	f7ff ff13 	bl	8000d38 <checkerror>
 8000f12:	1c43      	adds	r3, r0, #1
 8000f14:	d0ec      	beq.n	8000ef0 <_swistat+0x18>
 8000f16:	6120      	str	r0, [r4, #16]
 8000f18:	2000      	movs	r0, #0
 8000f1a:	e7e9      	b.n	8000ef0 <_swistat+0x18>

08000f1c <_fstat>:
 8000f1c:	b570      	push	{r4, r5, r6, lr}
 8000f1e:	000c      	movs	r4, r1
 8000f20:	0005      	movs	r5, r0
 8000f22:	2258      	movs	r2, #88	; 0x58
 8000f24:	2100      	movs	r1, #0
 8000f26:	0020      	movs	r0, r4
 8000f28:	f7ff f98c 	bl	8000244 <memset>
 8000f2c:	0028      	movs	r0, r5
 8000f2e:	0021      	movs	r1, r4
 8000f30:	f7ff ffd2 	bl	8000ed8 <_swistat>
 8000f34:	bd70      	pop	{r4, r5, r6, pc}

08000f36 <_stat>:
 8000f36:	b570      	push	{r4, r5, r6, lr}
 8000f38:	000d      	movs	r5, r1
 8000f3a:	0004      	movs	r4, r0
 8000f3c:	2258      	movs	r2, #88	; 0x58
 8000f3e:	2100      	movs	r1, #0
 8000f40:	0028      	movs	r0, r5
 8000f42:	f7ff f97f 	bl	8000244 <memset>
 8000f46:	0020      	movs	r0, r4
 8000f48:	2100      	movs	r1, #0
 8000f4a:	f000 f813 	bl	8000f74 <_swiopen>
 8000f4e:	0004      	movs	r4, r0
 8000f50:	1c43      	adds	r3, r0, #1
 8000f52:	d00c      	beq.n	8000f6e <_stat+0x38>
 8000f54:	2381      	movs	r3, #129	; 0x81
 8000f56:	686a      	ldr	r2, [r5, #4]
 8000f58:	021b      	lsls	r3, r3, #8
 8000f5a:	4313      	orrs	r3, r2
 8000f5c:	0029      	movs	r1, r5
 8000f5e:	606b      	str	r3, [r5, #4]
 8000f60:	f7ff ffba 	bl	8000ed8 <_swistat>
 8000f64:	0005      	movs	r5, r0
 8000f66:	0020      	movs	r0, r4
 8000f68:	f7ff ff90 	bl	8000e8c <_close>
 8000f6c:	002c      	movs	r4, r5
 8000f6e:	0020      	movs	r0, r4
 8000f70:	bd70      	pop	{r4, r5, r6, pc}
	...

08000f74 <_swiopen>:
 8000f74:	b5f0      	push	{r4, r5, r6, r7, lr}
 8000f76:	000d      	movs	r5, r1
 8000f78:	2600      	movs	r6, #0
 8000f7a:	b099      	sub	sp, #100	; 0x64
 8000f7c:	9000      	str	r0, [sp, #0]
 8000f7e:	00f3      	lsls	r3, r6, #3
 8000f80:	9301      	str	r3, [sp, #4]
 8000f82:	4b29      	ldr	r3, [pc, #164]	; (8001028 <_swiopen+0xb4>)
 8000f84:	00f2      	lsls	r2, r6, #3
 8000f86:	589c      	ldr	r4, [r3, r2]
 8000f88:	1c63      	adds	r3, r4, #1
 8000f8a:	d038      	beq.n	8000ffe <_swiopen+0x8a>
 8000f8c:	3601      	adds	r6, #1
 8000f8e:	2e14      	cmp	r6, #20
 8000f90:	d1f5      	bne.n	8000f7e <_swiopen+0xa>
 8000f92:	f7ff f92d 	bl	80001f0 <__errno>
 8000f96:	2401      	movs	r4, #1
 8000f98:	2318      	movs	r3, #24
 8000f9a:	4264      	negs	r4, r4
 8000f9c:	6003      	str	r3, [r0, #0]
 8000f9e:	e03f      	b.n	8001020 <_swiopen+0xac>
 8000fa0:	2302      	movs	r3, #2
 8000fa2:	03ec      	lsls	r4, r5, #15
 8000fa4:	0fe4      	lsrs	r4, r4, #31
 8000fa6:	421d      	tst	r5, r3
 8000fa8:	d000      	beq.n	8000fac <_swiopen+0x38>
 8000faa:	431c      	orrs	r4, r3
 8000fac:	4b1f      	ldr	r3, [pc, #124]	; (800102c <_swiopen+0xb8>)
 8000fae:	421d      	tst	r5, r3
 8000fb0:	d001      	beq.n	8000fb6 <_swiopen+0x42>
 8000fb2:	2304      	movs	r3, #4
 8000fb4:	431c      	orrs	r4, r3
 8000fb6:	2308      	movs	r3, #8
 8000fb8:	421d      	tst	r5, r3
 8000fba:	d002      	beq.n	8000fc2 <_swiopen+0x4e>
 8000fbc:	2204      	movs	r2, #4
 8000fbe:	4394      	bics	r4, r2
 8000fc0:	431c      	orrs	r4, r3
 8000fc2:	9b00      	ldr	r3, [sp, #0]
 8000fc4:	0018      	movs	r0, r3
 8000fc6:	9302      	str	r3, [sp, #8]
 8000fc8:	f7ff f89e 	bl	8000108 <strlen>
 8000fcc:	607c      	str	r4, [r7, #4]
 8000fce:	60b8      	str	r0, [r7, #8]
 8000fd0:	2401      	movs	r4, #1
 8000fd2:	1c20      	adds	r0, r4, #0
 8000fd4:	1c39      	adds	r1, r7, #0
 8000fd6:	beab      	bkpt	0x00ab
 8000fd8:	1c04      	adds	r4, r0, #0
 8000fda:	2c00      	cmp	r4, #0
 8000fdc:	db0a      	blt.n	8000ff4 <_swiopen+0x80>
 8000fde:	4b12      	ldr	r3, [pc, #72]	; (8001028 <_swiopen+0xb4>)
 8000fe0:	00f2      	lsls	r2, r6, #3
 8000fe2:	509c      	str	r4, [r3, r2]
 8000fe4:	0013      	movs	r3, r2
 8000fe6:	4a10      	ldr	r2, [pc, #64]	; (8001028 <_swiopen+0xb4>)
 8000fe8:	0034      	movs	r4, r6
 8000fea:	4694      	mov	ip, r2
 8000fec:	2200      	movs	r2, #0
 8000fee:	4463      	add	r3, ip
 8000ff0:	605a      	str	r2, [r3, #4]
 8000ff2:	e015      	b.n	8001020 <_swiopen+0xac>
 8000ff4:	0020      	movs	r0, r4
 8000ff6:	f7ff fe91 	bl	8000d1c <error>
 8000ffa:	0004      	movs	r4, r0
 8000ffc:	e010      	b.n	8001020 <_swiopen+0xac>
 8000ffe:	23a0      	movs	r3, #160	; 0xa0
 8001000:	002a      	movs	r2, r5
 8001002:	011b      	lsls	r3, r3, #4
 8001004:	401a      	ands	r2, r3
 8001006:	af02      	add	r7, sp, #8
 8001008:	429a      	cmp	r2, r3
 800100a:	d1c9      	bne.n	8000fa0 <_swiopen+0x2c>
 800100c:	0039      	movs	r1, r7
 800100e:	9800      	ldr	r0, [sp, #0]
 8001010:	f7ff ff91 	bl	8000f36 <_stat>
 8001014:	1c43      	adds	r3, r0, #1
 8001016:	d0c3      	beq.n	8000fa0 <_swiopen+0x2c>
 8001018:	f7ff f8ea 	bl	80001f0 <__errno>
 800101c:	2311      	movs	r3, #17
 800101e:	6003      	str	r3, [r0, #0]
 8001020:	0020      	movs	r0, r4
 8001022:	b019      	add	sp, #100	; 0x64
 8001024:	bdf0      	pop	{r4, r5, r6, r7, pc}
 8001026:	46c0      	nop			; (mov r8, r8)
 8001028:	200000a8 	.word	0x200000a8
 800102c:	00000601 	.word	0x00000601

08001030 <_get_semihosting_exts>:
 8001030:	b5f0      	push	{r4, r5, r6, r7, lr}
 8001032:	b085      	sub	sp, #20
 8001034:	9000      	str	r0, [sp, #0]
 8001036:	9101      	str	r1, [sp, #4]
 8001038:	4827      	ldr	r0, [pc, #156]	; (80010d8 <_get_semihosting_exts+0xa8>)
 800103a:	2100      	movs	r1, #0
 800103c:	0015      	movs	r5, r2
 800103e:	f7ff ff99 	bl	8000f74 <_swiopen>
 8001042:	0004      	movs	r4, r0
 8001044:	002a      	movs	r2, r5
 8001046:	2100      	movs	r1, #0
 8001048:	9800      	ldr	r0, [sp, #0]
 800104a:	f7ff f8fb 	bl	8000244 <memset>
 800104e:	1c63      	adds	r3, r4, #1
 8001050:	d015      	beq.n	800107e <_get_semihosting_exts+0x4e>
 8001052:	0020      	movs	r0, r4
 8001054:	f7ff fe48 	bl	8000ce8 <findslot>
 8001058:	260c      	movs	r6, #12
 800105a:	0007      	movs	r7, r0
 800105c:	1c30      	adds	r0, r6, #0
 800105e:	1c39      	adds	r1, r7, #0
 8001060:	beab      	bkpt	0x00ab
 8001062:	1c06      	adds	r6, r0, #0
 8001064:	0030      	movs	r0, r6
 8001066:	f7ff fe67 	bl	8000d38 <checkerror>
 800106a:	2803      	cmp	r0, #3
 800106c:	dd02      	ble.n	8001074 <_get_semihosting_exts+0x44>
 800106e:	3803      	subs	r0, #3
 8001070:	42a8      	cmp	r0, r5
 8001072:	dc07      	bgt.n	8001084 <_get_semihosting_exts+0x54>
 8001074:	0020      	movs	r0, r4
 8001076:	2401      	movs	r4, #1
 8001078:	f7ff ff08 	bl	8000e8c <_close>
 800107c:	4264      	negs	r4, r4
 800107e:	0020      	movs	r0, r4
 8001080:	b005      	add	sp, #20
 8001082:	bdf0      	pop	{r4, r5, r6, r7, pc}
 8001084:	ae03      	add	r6, sp, #12
 8001086:	2204      	movs	r2, #4
 8001088:	0031      	movs	r1, r6
 800108a:	0020      	movs	r0, r4
 800108c:	f7ff fe6a 	bl	8000d64 <_read>
 8001090:	2803      	cmp	r0, #3
 8001092:	ddef      	ble.n	8001074 <_get_semihosting_exts+0x44>
 8001094:	7833      	ldrb	r3, [r6, #0]
 8001096:	2b53      	cmp	r3, #83	; 0x53
 8001098:	d1ec      	bne.n	8001074 <_get_semihosting_exts+0x44>
 800109a:	7873      	ldrb	r3, [r6, #1]
 800109c:	2b48      	cmp	r3, #72	; 0x48
 800109e:	d1e9      	bne.n	8001074 <_get_semihosting_exts+0x44>
 80010a0:	78b3      	ldrb	r3, [r6, #2]
 80010a2:	2b46      	cmp	r3, #70	; 0x46
 80010a4:	d1e6      	bne.n	8001074 <_get_semihosting_exts+0x44>
 80010a6:	78f3      	ldrb	r3, [r6, #3]
 80010a8:	2b42      	cmp	r3, #66	; 0x42
 80010aa:	d1e3      	bne.n	8001074 <_get_semihosting_exts+0x44>
 80010ac:	2201      	movs	r2, #1
 80010ae:	0020      	movs	r0, r4
 80010b0:	9901      	ldr	r1, [sp, #4]
 80010b2:	f7ff fe71 	bl	8000d98 <_swilseek>
 80010b6:	2800      	cmp	r0, #0
 80010b8:	dbdc      	blt.n	8001074 <_get_semihosting_exts+0x44>
 80010ba:	002a      	movs	r2, r5
 80010bc:	9900      	ldr	r1, [sp, #0]
 80010be:	0020      	movs	r0, r4
 80010c0:	f7ff fe50 	bl	8000d64 <_read>
 80010c4:	0005      	movs	r5, r0
 80010c6:	0020      	movs	r0, r4
 80010c8:	f7ff fee0 	bl	8000e8c <_close>
 80010cc:	0028      	movs	r0, r5
 80010ce:	f7ff fe33 	bl	8000d38 <checkerror>
 80010d2:	0004      	movs	r4, r0
 80010d4:	e7d3      	b.n	800107e <_get_semihosting_exts+0x4e>
 80010d6:	46c0      	nop			; (mov r8, r8)
 80010d8:	080012a0 	.word	0x080012a0

080010dc <initialise_semihosting_exts>:
 80010dc:	b5f7      	push	{r0, r1, r2, r4, r5, r6, r7, lr}
 80010de:	2401      	movs	r4, #1
 80010e0:	2100      	movs	r1, #0
 80010e2:	4e09      	ldr	r6, [pc, #36]	; (8001108 <initialise_semihosting_exts+0x2c>)
 80010e4:	4d09      	ldr	r5, [pc, #36]	; (800110c <initialise_semihosting_exts+0x30>)
 80010e6:	af01      	add	r7, sp, #4
 80010e8:	0022      	movs	r2, r4
 80010ea:	0038      	movs	r0, r7
 80010ec:	6031      	str	r1, [r6, #0]
 80010ee:	602c      	str	r4, [r5, #0]
 80010f0:	f7ff ff9e 	bl	8001030 <_get_semihosting_exts>
 80010f4:	2800      	cmp	r0, #0
 80010f6:	dd05      	ble.n	8001104 <initialise_semihosting_exts+0x28>
 80010f8:	2202      	movs	r2, #2
 80010fa:	783b      	ldrb	r3, [r7, #0]
 80010fc:	401c      	ands	r4, r3
 80010fe:	4013      	ands	r3, r2
 8001100:	6034      	str	r4, [r6, #0]
 8001102:	602b      	str	r3, [r5, #0]
 8001104:	bdf7      	pop	{r0, r1, r2, r4, r5, r6, r7, pc}
 8001106:	46c0      	nop			; (mov r8, r8)
 8001108:	20000064 	.word	0x20000064
 800110c:	20000068 	.word	0x20000068

08001110 <_has_ext_stdout_stderr>:
 8001110:	b510      	push	{r4, lr}
 8001112:	4c04      	ldr	r4, [pc, #16]	; (8001124 <_has_ext_stdout_stderr+0x14>)
 8001114:	6823      	ldr	r3, [r4, #0]
 8001116:	2b00      	cmp	r3, #0
 8001118:	da01      	bge.n	800111e <_has_ext_stdout_stderr+0xe>
 800111a:	f7ff ffdf 	bl	80010dc <initialise_semihosting_exts>
 800111e:	6820      	ldr	r0, [r4, #0]
 8001120:	bd10      	pop	{r4, pc}
 8001122:	46c0      	nop			; (mov r8, r8)
 8001124:	20000068 	.word	0x20000068

08001128 <initialise_monitor_handles>:
 8001128:	b5f0      	push	{r4, r5, r6, r7, lr}
 800112a:	4b27      	ldr	r3, [pc, #156]	; (80011c8 <initialise_monitor_handles+0xa0>)
 800112c:	b085      	sub	sp, #20
 800112e:	9301      	str	r3, [sp, #4]
 8001130:	2500      	movs	r5, #0
 8001132:	2303      	movs	r3, #3
 8001134:	ac01      	add	r4, sp, #4
 8001136:	60a3      	str	r3, [r4, #8]
 8001138:	2701      	movs	r7, #1
 800113a:	6065      	str	r5, [r4, #4]
 800113c:	1c38      	adds	r0, r7, #0
 800113e:	1c21      	adds	r1, r4, #0
 8001140:	beab      	bkpt	0x00ab
 8001142:	1c07      	adds	r7, r0, #0
 8001144:	2101      	movs	r1, #1
 8001146:	4b21      	ldr	r3, [pc, #132]	; (80011cc <initialise_monitor_handles+0xa4>)
 8001148:	4249      	negs	r1, r1
 800114a:	601f      	str	r7, [r3, #0]
 800114c:	002b      	movs	r3, r5
 800114e:	4d20      	ldr	r5, [pc, #128]	; (80011d0 <initialise_monitor_handles+0xa8>)
 8001150:	00da      	lsls	r2, r3, #3
 8001152:	3301      	adds	r3, #1
 8001154:	50a9      	str	r1, [r5, r2]
 8001156:	2b14      	cmp	r3, #20
 8001158:	d1fa      	bne.n	8001150 <initialise_monitor_handles+0x28>
 800115a:	f7ff ffd9 	bl	8001110 <_has_ext_stdout_stderr>
 800115e:	2800      	cmp	r0, #0
 8001160:	d018      	beq.n	8001194 <initialise_monitor_handles+0x6c>
 8001162:	4b19      	ldr	r3, [pc, #100]	; (80011c8 <initialise_monitor_handles+0xa0>)
 8001164:	2701      	movs	r7, #1
 8001166:	9301      	str	r3, [sp, #4]
 8001168:	2303      	movs	r3, #3
 800116a:	60a3      	str	r3, [r4, #8]
 800116c:	3301      	adds	r3, #1
 800116e:	6063      	str	r3, [r4, #4]
 8001170:	1c38      	adds	r0, r7, #0
 8001172:	1c21      	adds	r1, r4, #0
 8001174:	beab      	bkpt	0x00ab
 8001176:	1c06      	adds	r6, r0, #0
 8001178:	4b16      	ldr	r3, [pc, #88]	; (80011d4 <initialise_monitor_handles+0xac>)
 800117a:	4a13      	ldr	r2, [pc, #76]	; (80011c8 <initialise_monitor_handles+0xa0>)
 800117c:	601e      	str	r6, [r3, #0]
 800117e:	2303      	movs	r3, #3
 8001180:	9201      	str	r2, [sp, #4]
 8001182:	60a3      	str	r3, [r4, #8]
 8001184:	3305      	adds	r3, #5
 8001186:	6063      	str	r3, [r4, #4]
 8001188:	1c38      	adds	r0, r7, #0
 800118a:	1c21      	adds	r1, r4, #0
 800118c:	beab      	bkpt	0x00ab
 800118e:	1c04      	adds	r4, r0, #0
 8001190:	4b11      	ldr	r3, [pc, #68]	; (80011d8 <initialise_monitor_handles+0xb0>)
 8001192:	601c      	str	r4, [r3, #0]
 8001194:	4f10      	ldr	r7, [pc, #64]	; (80011d8 <initialise_monitor_handles+0xb0>)
 8001196:	683b      	ldr	r3, [r7, #0]
 8001198:	3301      	adds	r3, #1
 800119a:	d102      	bne.n	80011a2 <initialise_monitor_handles+0x7a>
 800119c:	4b0d      	ldr	r3, [pc, #52]	; (80011d4 <initialise_monitor_handles+0xac>)
 800119e:	681b      	ldr	r3, [r3, #0]
 80011a0:	603b      	str	r3, [r7, #0]
 80011a2:	2400      	movs	r4, #0
 80011a4:	4b09      	ldr	r3, [pc, #36]	; (80011cc <initialise_monitor_handles+0xa4>)
 80011a6:	606c      	str	r4, [r5, #4]
 80011a8:	681b      	ldr	r3, [r3, #0]
 80011aa:	602b      	str	r3, [r5, #0]
 80011ac:	f7ff ffb0 	bl	8001110 <_has_ext_stdout_stderr>
 80011b0:	42a0      	cmp	r0, r4
 80011b2:	d006      	beq.n	80011c2 <initialise_monitor_handles+0x9a>
 80011b4:	4b07      	ldr	r3, [pc, #28]	; (80011d4 <initialise_monitor_handles+0xac>)
 80011b6:	60ec      	str	r4, [r5, #12]
 80011b8:	681b      	ldr	r3, [r3, #0]
 80011ba:	616c      	str	r4, [r5, #20]
 80011bc:	60ab      	str	r3, [r5, #8]
 80011be:	683b      	ldr	r3, [r7, #0]
 80011c0:	612b      	str	r3, [r5, #16]
 80011c2:	b005      	add	sp, #20
 80011c4:	bdf0      	pop	{r4, r5, r6, r7, pc}
 80011c6:	46c0      	nop			; (mov r8, r8)
 80011c8:	080012b6 	.word	0x080012b6
 80011cc:	200000a0 	.word	0x200000a0
 80011d0:	200000a8 	.word	0x200000a8
 80011d4:	200000a4 	.word	0x200000a4
 80011d8:	2000009c 	.word	0x2000009c

080011dc <_isatty>:
 80011dc:	b570      	push	{r4, r5, r6, lr}
 80011de:	f7ff fd83 	bl	8000ce8 <findslot>
 80011e2:	2509      	movs	r5, #9
 80011e4:	1e04      	subs	r4, r0, #0
 80011e6:	d104      	bne.n	80011f2 <_isatty+0x16>
 80011e8:	f7ff f802 	bl	80001f0 <__errno>
 80011ec:	6005      	str	r5, [r0, #0]
 80011ee:	0020      	movs	r0, r4
 80011f0:	bd70      	pop	{r4, r5, r6, pc}
 80011f2:	1c28      	adds	r0, r5, #0
 80011f4:	1c21      	adds	r1, r4, #0
 80011f6:	beab      	bkpt	0x00ab
 80011f8:	1c04      	adds	r4, r0, #0
 80011fa:	0020      	movs	r0, r4
 80011fc:	2c01      	cmp	r4, #1
 80011fe:	d0f7      	beq.n	80011f0 <_isatty+0x14>
 8001200:	f7fe fff6 	bl	80001f0 <__errno>
 8001204:	2400      	movs	r4, #0
 8001206:	0005      	movs	r5, r0
 8001208:	2613      	movs	r6, #19
 800120a:	1c30      	adds	r0, r6, #0
 800120c:	1c21      	adds	r1, r4, #0
 800120e:	beab      	bkpt	0x00ab
 8001210:	1c06      	adds	r6, r0, #0
 8001212:	602e      	str	r6, [r5, #0]
 8001214:	e7eb      	b.n	80011ee <_isatty+0x12>
	...

08001218 <_init>:
 8001218:	b5f8      	push	{r3, r4, r5, r6, r7, lr}
 800121a:	46c0      	nop			; (mov r8, r8)
 800121c:	bcf8      	pop	{r3, r4, r5, r6, r7}
 800121e:	bc08      	pop	{r3}
 8001220:	469e      	mov	lr, r3
 8001222:	4770      	bx	lr

08001224 <_fini>:
 8001224:	b5f8      	push	{r3, r4, r5, r6, r7, lr}
 8001226:	46c0      	nop			; (mov r8, r8)
 8001228:	bcf8      	pop	{r3, r4, r5, r6, r7}
 800122a:	bc08      	pop	{r3}
 800122c:	469e      	mov	lr, r3
 800122e:	4770      	bx	lr
